:020000040000FA
:5C000000FFFF62D73700FFFFFFFFFFFFFFFFFFFFFFFFFFFFFFFFFFFFFFFFFFFFFFFFFFFFFFFFFFFFFFFFFFFFFFFFFFFFFFFFFFFFFFFFFFFFFFFFFFFFFFFFFFFFFFFFFFFFFFFFFFFFFFFFFFFFFFFFFFFFFFFFFFFFFFFFFFFFFFFFFFFFFFFFFFFF8C
:5C005C00800CB001324006D8001960036C800CB00136C026C8069800036C006C90012610049800190802412008040100000000400684001B10026C800CB00132C006824010001360026C800D100482401008021B20036C300106043240101CFDFD
:5C00B8000016400258000B20012C8004900016400248000D6001348004900012C00254800A50012C4005A80015A00200000000000B5001244005900016400258000950012A8006D000124002A80015A002548004500112A002B40015A0027CFE53
:5C01140000000400000000020000080001000004800010000010000000010000010000100000000008000120000400000000000000024000080001000004000010000240000000000000012000048000100002400000000100000400001060FF91
:5C01700000000400000000020000080001000004800010000010000000010000010000100000000008000120000400000000000000024000080001000004000010000240000000000000012000048000100002400000000100000400001060FF35
:5C01CC00000020000580001000024000080001200005800000020000000800202000000000000000000000000000000000000080000000020000080000200000800000000000000000200004000000000000000800002000000000000000ACFFC7
:5C0228000000A0001080005000004000080000A00010800088000000000880000000000000000000000000000000000084000000000000020000080000A0000080000000000000008000100100000000000020000080000000000000000014FF80
:5C0284000000000020000000000000000000000001000004000010000000000000000000000000000000400000000000000000000000000000000000000000000000800010000000000800002000040000000002000000000000000002001CFCD1
:5C02E000000000000008000000000000000000004000000001000004000000000000000000000000000000100000000000000000000000000000000000000000000000200004000000000210000800010000008000000000000000000000E8FDC1
:5C033C000000008001000000000000000000000C0000300000C00000000000000000000000000000000003000000000000000000000000000000000000000000000006C00000000060000C800130000000001800000000000000000006204CFE7A
:5C039800000000800000000000000000000000040000100000400000000000000000000000000000000001000000000000000000000000000000000000000000000002400000000020000480001000000000080000000000000000005A0030FFAD
:5C03F400000000001602000000000000000000300100C0080000130000000000000000000000000000002C020000000000000000000000000000000000000000000058000B0000008091302216C04000000060020000000000000000000178FDA7
:5C045000000000000700000000000000000000380800E0400080830000000000000000000000000000000E00000000000000000000000000000000000000000000001C8403040000C001380007E200000000701000000000000000001C1060FD46
:5C04AC00000000000600000000000000000000300000C0000000030000000000000000000000000000000C00000000000000000000000000000000000000000000001800030000008001300006C00000000060000000000000000000180050FD98
:5C050800000000000600000000000000000000300000C0000000030000000000000000000000000000000C00000000000000000000000000000000000000000000001800030000008001300006C00000000060000000000000000000981058FCA4
:5C056400040000002010000000000000000000040000000480001000000000000400000000000000000040000004000000000000000200000800000000000000000080400000000080213082000004024000080001000000012000000080E6FE36
:5C05C00000000000000800000000000000000000000000000120000400000000000000000000000000000010000000000000000000000000000000000000000000000020000000000000004000000001000000000000000040000800000088FE73
:5C061C000800008001300001000000000000000C0000300006C00000000000000C0000000000000000000300000C000000000000000620001880000000000000000006C000000000E0013C8001300006C00018000300000C800100000000D9FD15
:5C0678000000008000D0020000000000000000040000100002400000000000000400000000000000000001000004000000000000005A000068010000000000000000024000000000A081349000100002400008000100000480000000008001FE2D
:5C06D400040000004600020000000000000000302100C0021801A30000000000300900000000000000004C02003010000000000000800400000200000000000000009800030000008051B00016C28818200360120C000030092601000000A1FF2D
:5C0730000000000007E4800000000000000000380000E0001DA0030000000000380000000000000000000E000038000000000000001C0000701000000000000000001C8403010000C001384007E0001C800372000E10003800070000000020FCC2
:5C078C000800000006C0000000000000000000300000C0001800030000000000300000000000000000000C00003000000000000000180000600000000000000000001800030000008001300006C00018000360000C00003000060000008024FF62
:5C07E8000000000006C0800000000000000000300000C0001800030000000000300000000000000000000C00003000000000000000580400602000000000000000001800030000008051300906C00018000360000C000030000600000000A0FDD7
:5C08440004000000200004000010000000000000010000040240000000000000000000000000000000004000000000000000000000020000080001000000000000040240000800002000048000C0088040000002010000048000000000800EFD02
:5C08A00000000000000800010000040000000000400000000100000000000000000000000000000000000010000000000000000000000000000000000000000000000100000000000000000000000001200000800000000000000000000034FDCB
:5C08FC000800008001300000C00000000000000C0000300006C00000000000000000000000000000000003000000000000000000000620001800030000000000300006C00018000060800CC001F00006C00018000300000C80010000000071FC5B
:5C095800000000800010000040000000000000040000100002400000000000000000000000000000000001000000000000000000005A000008000100000000001000024000080000A011B48000D024024000080001000004800000000080CDFC6E
:5C09B40004000000C6C00000000B0200000000300200C0005804030000000000000000000000000000000C0000000000000000000000010060142C0000000000C0025800236044000010000146C00898042360128C0000B010060400000059FC76
:5C0A10000000000007E0000180030000000000380800E0001D80030200000000000000000000000000000E040000000000000000001C100070000E1000000000E0801C8883700000C041384007E1201C808370000E020038000700000000B0FD8E
:5C0A6C000800000006C0000000030000000000300000C0001800030000000000000000000000000000000C0000000000000000000018000060000C0000000000C0001800036000008041300806C00018000360000C0000300006000000806CFE21
:5C0AC8000000000006C0000000030000000000300000C0001800030000000000000000000000000000000C0000000000000000000058200060000C0000000000C0001800036000008011300106C02818000360000C000030000600000000A8FEC0
:5C0B2400040000004610000000430000000008040000C0108040000000000000040000000000000000008C000000000000000000008000006004010000000000000002001000000000080400200004020010080040000000012000000080CCFCC2
:5C0B8000000000000008000000000000000000020000000000200000000000000000000000000000000000100000000000000000000020000080000000000000000000000004000000000200000800010000040000100000400008000000C8FC10
:5C0BDC000800008007300000C00300000060000C0000F00006C00000000000000C0000000000000000000F000000000000000000000600007820030000000000000006C00000000060000CC001300006C00018000300000C800100000000F5FCDB
:5C0C38000000008016140000408B0000002000040000D0240240000000000000040000000000000000004D02000000000000000000020000680101000000000000000240000000002000B48000100002400008000100000480000000000060FFFE
:5C0C94000400000016C0080100030000008051B04000C0085804A30000000000300000000000000000008C0000000000000000000058080060102C0800000000000058000B0000008001001016C24298040B60044C0200B0084601000080E8FF09
:5C0CF0000000000007E100008003010000C001380000E0201C80030000000000381000000000000000000E080000000000000000001C000070000E000000000000001C8483000000C0013A0007E0001C808370100E00003800070000000014FCAB
:5C0D4C000800000006C0000000830000008001300000C0001800030000000000300000000000000000000C0800000000000000000018000060100C000000000000001800030000008001300806C00018000360000C00003000060000000091FFAF
:5C0DA8000000000026C2000000230000008001300000C0221800030000000000300000000000000000002C0000000000000000000018000060040C000000000000001800030000008001300206C00018000360000C000030000600000000E0FF22
:5C0E040004000080000004000010000000200004000010008040000800010000040000000000000000000100000000000000000000180100000240000000800000001801230000002000040046000402001008000100000480000000008024FF31
:5C0E6000000000000000000100000400000000000000000000200000000000000000000000000000000000000000000000000000000020000080001000000000000000200004000000000000000800010000040000000000000000000000DCFC58
:5C0EBC000800008001380000C00000000060000C0000300007C00018000300000C00000000000000000003000000000000000000001E0000180003000000800100001EC00304000060800CC007300006C00018000300000C80010000000051FE8D
:5C0F1800000000801610000040000000002000040000D00202400008000100000400000000000000000001000000000000000000001A0500080001000000800000009A4403000000A011B480261100024000080001000004800000000000ACFC35
:5C0F74000400000020C0040000030100008051300200000858001360118C0000300100000000000000008C0000000000000000000018050060144C0000000006020018080300000000040106C6C02858200360142C000030102604000080FCFE45
:5C0FD0000000000007E180008003000000C001380800E0001D848370000E0800381000000000000000000E040000000000000000001C000070000E020000000700001C8083000000C001380007E0001C800371000E020038000700000000F8FC00
:5C102C000800000006C1000000030000008001300000C02018000360000C0000300000000000000000000C0000000000000000000018040060000C000000000600001800830000008001300806C00018000360000C00003000060000000089FE56
:5C1088000000000026C0000000030000008001300000C00218000360000C0000300000000000000000000C0000000000000000000058000060000C0000000006000098080B0000008001320046C10018000360000C00003000060000000004FEFF
:5C10E4000000040046C008000010000000000804000010000240000800000000008100000000000000000100000000000000000000800000080001000000000000001801100000008021040020C00818024300024000000400200000008074FEB2
:5C1140000000000000080001000004000000000200000000000000000000000000400000000000000000000000000000000000000000200000000000000000000000002000040000000000000008000100000080001000000000080000001CFF04
:5C119C0000000CC007F02000C00000000060000C0000300007C00018000000000C8001000000000000000300000000000000000000060000188003000000000000001EC000000000E0010E8001F0401EC00318000300000C80010000000039FD6B
:5C11F8000800B48006D1080040000000002000040000D0020240000800000000048000000000000000000100000000000000000000020000680101000000000000001A4400000000A005048000D0001A60030C000100000480000000000074FD39
:5C1254000000001016C0280000A30000008049300100000418110B6042000000300116020000000000004C0200000000000000000098100000002C000000000000009800230000008041000216C08418051360048C000030121600000080A8FDD9
:5C12B0000000380007E800008003000000C001380800E0201C80837000000000380807000000000000000E000000000000000000001C000070400E020000000000001C9083000000C001080807E1001C808370100E020038000701000000ACFFF5
:5C130C000400300006C0000000030000008001300000C0201800036000000000300006000000000000000C0000000000000000000018000060000C000000000000001808030000008001304006C02018008360000C00003000060000000011FD71
:5C1368000000301026C1220000030000008001300000C0001800036000000000300006000000000000000C0000000000000000000018000060100C000000000000001800030000008049B00006C00858042360000C00003000060000000004FF95
:5C13C40014000080000004024000080000200000810010000240000002000000000100000000000000008C00000000000000000000800000080001000000000000000200230000000008040020100080001008004000003082000000000020FDD8
:5C142000000000000000000100000000000000004000000000000000800000000040000000000000000000100000000000000000000020000000000000000000000000000004000000000200000800002000040000100000400000000000B0FC11
:5C147C000800008001300006C00018000060000C8001300006C00018000000000C0000000000000000000F000000000000000000000600001800030000000000000006E00304000060000CC001300006C00018000300003C80010000000050FE10
:5C14D8000C000080001000024000080000200004800010000240000800000000040000000000000000000D02000000000000000000020000080001000000000000005A40130000002000B480001000024000080001000034880000000000D9FCC9
:5C1534000800000010C1045810236041008001300046001858000B6112000000300900000000000000002C0000000000000000000018100060014C000000000000008004130000008001820046C00818012360002C000030011602000000D4FCAA
:5C1590000000000001E0201C8003740000C0013A400724001C84037000000000380000000000000000000E020000000000000000001C000070800E020000000000001C8003020000C001382007E1801C848370200E02003808070000000064FF7F
:5C15EC000400000006C8001800036000008001300006C0001900036000000000300000000000000000000C0000000000000000000018000060000C000000000000001810030000008001300806C00018000360000C0000300806000000809CFE1A
:5C1648000000000016C0001800036000008001300006C0021800036000000000300000000000000000002C0400000000000000000018000060000C000000000000001801A30000008001B00006C00018000360000C0000300106000000002CFD83
:5C16A40024000080001000004000000001200030020010001802100002002000040000000000400008000100080000000000000000020000000240000000000000000240000000010008048000100002400000020120000001460000008074FC33
:5C17000000000000000000000000000000000000400000000000000480000000000000000000000000000000000200000000000000000000008000100000000000000000000000000000020000000000000000800000000040000800000068FC09
:5C175C006800008001380001C00000000360003C000030001FC00018000060000C0000000000C000180003600000000000000000000620001800030000000000000006E00000000360000CC001380006C00018000360000C800700000000E9FE98
:5C17B8002000008016D0020040000000012000340900D0021A440008000020000400000000004000080001200000000000000000005A0000080001000000000000005A40000000012000B4801610000240000800012000048046010000003CFC04
:5C181400840500000008220000A300008C8149300A00008498040B6011008009300100000000000B60842C8209010000000000000000030060442C0000000000000040040B00000C8109000120C12818010B60144C8231B000160100008074FD84
:5C187000C001020007E00000800300000EC001380000E0001C8083700000C0013A0800000000800371000EC00100000000000000001C000070000E020000000000001C808300000EC081381007E0001C848370000EC00138080700000000BCFE17
:5C18CC008801000006C10000000300000C8001300000C0201800036000008001300000000000000360000C8001000000000000000018000060000C0000000000000018040300000C8001304006C00018000360000C80013000060000000025FEED
:5C1928008001000006C02000000300000C8001B00800C0085810036000008001300000000000000360000C8001000000000000000018040060000C0000000000000018000300000C8001300226C40018000360000C800130000601000000ACFD4C
:5C19840004000000000000000000000000000000000000000000000000000000000000000000000000000000000000000000000000000000000000000000000000000000000000000000000000000000000000000000000000000000008050FF34
:5C19E000200004800010000240000800012000048000100002400008000120000480001000024000080001200004000000000010000240000800012000048000100002400008000120000480001000024000080001200004800010000200BCFCC3
:5C1A3C00080000000000000000000000000000000000000000000000000000000000000000000000000000000000000000000000000000000000000000000000000000000000000000000000000000000000000000000000000000000000C5FE83
:5C1A9800200004800010000240000800012000048000100002400008000120000480001000024000080001200004000000000010000240000800012000048000100002400008000120000480001000024000080001200004800010000200BCFC0A
:5C1AF400040120000480001000024000080001200004800010000240000800012000040000000002400008000120000000000000001000004000080000000004800010000240000800012000048000100002400008000120000400001080C0FF5B
:5C1B50000000000000000000000000000000000000000000000000000000000000000010000200000000000000000000000000100000400000000020000400000000000000000000000000000000000000000000000000000000100000008CFE19
:5C1BAC008800100002400008000120000480001000024000080001200004800010000200000000012000048000100000000000000008000020000400000000024000080001200004800010000240000800012000048000100002000008008DFED1
:5C1C08000000000000000000000000000000000000000000000000000000000000000010000200000000000000000000000000100000400000000020000400000000000000000000000000000000000000000000000000000000100000008CFE60
:5C1C6400000000000000000000000000000000000000000000000000000000000000000000000000000000000000000000000000000000000000000000000000000000000000000000000000000000000000000000000000000000000000DCFF49
:5C1CC000000000000000000000000000000000000000000000000000000000000000000000000000000000000000000000000000000000000000000000000000000000000000000000000000000000000000000000000000000000000000DCFFED
:5C1D1C00000000000000000000000000000000000000000000000000000000000000000000000000000000000000000000000000000000000000000000000000000000000000000000000000000000000000000000000000000000000000DCFF90
:5C1D7800000000000000000000000000000000000000000000000000000000000000000000000000000000000000000000000000000000000000000000000000000000000000000000000000000000000000000000000000000000000000DCFF34
:5C1DD40000000000000000008000000001000000000000000000000000000000000000000000000000000000000800000000000000000000000000000000000000000000000000000080000000000000200000000000000000000000000064FC2A
:5C1E3000000000000800000000000000000000000000008000010000000000000000000000000000000008000000000000000000000000000000000000000000000000000000000000000000000000000000000000000000000000000000CCFEFB
:5C1E8C00000000000000000000000000000000000000000000000000000000000000000000000000000000000000000000000000000000000000000000000000000000000000000000000000000000000000000000000000000000000000DCFF1F
:5C1EE800000000000000000000000000000000000000000000000000000000000000000000000000000000000000000000000000000000000000000000000000000000000000000000000000000000000000000000000000000000000000DCFFC3
:5C1F4400000000000000000000000000000000000000000000000000000000000000000000000000000000000000000000000000000000000000000000000000000000000000000000000000000000000000000000000000000000000000DCFF66
:5C1FA000000000000000000000000000000000000000000000000000000000000000000000000000000000000000000000000000000000000000000000000000000000000000000000000000000000000000000000000000000000000000DCFF0A
:5C1FFC00000000000000000000000000000000000000100000000000000000000000000000000000000000000000000000000000000000000000000000000000000000008000000000002000000000000000000000000000000000000000E4FDF8
:5C205800000000000004000000000000000000000000000000000000000000000000000000000000000000000000000000000000008010000000000000000000000000000000000000000000000000000000000000000000002000000000A5FDD6
:5C20B40004000000000000000000000000000000000000000000000000000000000000000000000000000000000000000000000000000000000000000000000000000000000000000000000000000000000000000000000000000000008050FFFD
:5C211000000000000000000000000000000000000000000000000000000000000000000000000000000000000000000000000000000000000000000000000000000000000000000000000000000000000040000000000000000000000000ABFC8C
:5C216C0000000000000000000000000000000010000000000000810000000000000000000000000000000000000000000000000000000000000000000000000000000000000000008000000000400000000020100080000020000000000498FF5B
:5C21C800000000000000000000000000000000000000000000000000000000000000000000000000000000000000000000000000000000010000000000000000000000000020000000000000000000000000000000000000000000000000CCFCD2
:5C22240000000000000000000000000000000008000000000080000100000000000000000000000000000000000000000000000000004000000000000000000000000000000800004000000000200000000010200040000010000000000804FFA2
:5C22800000000000000000000001000000000080000000000000890000000000000800800000000000000400000008000000000000000008000000000000000000000005800000000000040040010008000008000000040008000000000050FF27
:5C22DC00000000000000000000010000000000000000000000808000000000000008000000000000000004000000080000000000000000000000000000000000000000040001000000000000000100080000000000000000200000000000B0FFB4
:5C233800000000000000000000000000000000000000000000000000000000000000008000000000000000000000000000000000000000000000000000000000000000000000000000000000000000000000000000000000000000000000D4FFF6
:5C239400000000000000000000000000000000000000000000000000000000000000000000000000000000000000000000000000000000000000000000000000000000000000000000000000000000000000000000000000000000000000DCFF12
:5C23F000000000000000000000000000000000000000000000000000000000000000000000000000000000000000000000000000000000000000000000000000000000000000000100000000000000000000000000000000000000000000DCFEB6
:5C244C00000000000000000000000000000000000000000000000000000000000000000000000000000000000000000000000000000000000000000000000000000000000000000000000000000000000000040000000000000000000000D8FF59
:5C24A800000000000000000000000000000000020000000401000000000000000000000000000000000000000000000000000000000000000000000000000000000000000000000000000000000000000000000000000000000000000000A8FD2C
:5C250400000000000000000000000000000000000000000000000000000000002000000000000000000000000000000000000000000000000000000000000000000000000000000000000000000000000000000000000000000000000000DEFF7E
:5C256000000000000000000000000000000000000000000000000000000000000000000000000000000000000000000000000000000000000000000000000000000000000000000000000000000000000000000000000000000000000000DCFF44
:5C25BC00000000000000008000000000000000000000000000000000000000000000000000000000000000000000000000000000000000000000000000000000000000000000000000010000000000000000000000000000000000000000C4FE80
:5C261800000000000000000000000000000000000000000000000000000000000000000000000000000000000000000000000000000000000000000000000000000000000000000000000000000000000000000000000000000000000000DCFF8B
:5C267400000000000000000000000000000000000000000000000000000000000000000000000000000000000000000000000000000000008000000000000000000000000000000000000000000000000000000000000000000000000000D4FFB7
:5C26D00000000000000000000000000000000000000000000000000000000000000000000000000000000000000000000000000000000000004000000000000000000000000000000000000000000000000000000010000000000000000088FFD7
:5C272C00000000000000000000000000000000000000000000000000000000000000000000000000000000000000000000000000000000000000000000000000000000000000000000000000000000000000000000000000000000000000DCFF76
:5C27880000000000000000000000000000000000010000000000000000000000000000000000000000000000000000000000000000000000000000000000000000000000000000004000000000000000000000000000000000000000000098FE1E
:5C27E40000000000000000000000000000000000000000000000000000000000000000000000000000000000000000000000000000000000000000000000000000000000000000000000000000600000000000000000001800000000000078FCAD
:5C28400000000000000000000000000000000000000000000000000000000000000000000000000000000000000000000000000000000000000000000000000000001000000000000000001084000600000080000000000800000000000038FFD3
:5C289C00080000000201000000100002000000000000000000000100000000000000000000000000000000000000000000000000004A00000000000000000000000000002000000000004000000010000800000000000000001200000000C4FE2C
:5C28F8000000000000000800000000000000000000000000000000000000000040000000000000000000100000000000000000000000000000000000000000000000800004000000000002000000000000040000000000000000000000005CFC4A
:5C295400000000000000000000000000000000000000000000000000000001000100020000000000000000000000000000000000000000000000000000000001000000000000000000000000000000000000000000000000000000000000FCFC2A
:5C29B000000001000000000000000000000000000000000040000000000000000000000000000002001000000000000000000000000000000000000000000000000000000000000000000000000000000000000000000000000000000000B8FEC2
:5C2A0C0000000000000010000000000000000000100000000000000000000000000000000000000000000000000000000000000000000000000000000000000000000401000000000040008002000000040000000000000000000000000020FD66
:5C2A680000000000000000000000000000000000000000000000000000000000000000000000000000000000000000000000000000000000000000000000000000080000000000000000000000000000000000000000000000000000000054FFB7
:5C2AC4000000080000000000000004000000000000000001002000000000000000000000000000000000100100000000000000000000000000000000000000000000000000000000000A000000000000000000000000000000000000000220FC50
:5C2B200000000000000020000000000000000000400000000000400000000000000000000000000000000000000000000000000000000000000100000000000000002400800001000000000000000000000000000000000000000000000294FC81
:5C2B7C001A0000000000000000000000000000000000000000000000000000000000000000000000000000000000000000000000000000000000000000000000000000000000000000000000000000000000000000000000000000000040A0FD06
:5C2BD800000000000000000000000000000000000000000000000000000000000000000000000000000000000000000000000000000000000000000000000000000000000000000000000000000000000000000000000000000000000000DCFFC6
:5C2C340000000000001000008000080000000000080000800800400000008000000000000000000020000000000000000000000000000000000000020008000080000000810000000001000002000002040120000000000000000000000094FC77
:5C2C9000000000000000000000000000000000000000000000008000000400000000000000000000000000000010000000000000000040000000000000000000000000000000000100000000000000000000000000000000000000000000D4FF40
:5C2CEC000000A00000200000800010000000000010000040540000030A01400000000000000000001000000000040000000000000000400000000004280800A0200000800041010140050000010000048800100000000000000000000000E0FD80
:5C2D4800000080880880010005A2000084024110080080280800420002A0410420080004000840001001080000900000000000400004000000080400380000000000040000000100004400000241288804802011048250000C42010000007CFE0A
:5C2DA40000000008000000000480000004024010080000200800000000000000000800000002000000000000000400000000001000000000000004000000000000000000000000000040000002412008088020100482400020020100000000FC57
:5C2E0000000000000040000000010000008000000000400000008100000002001000000000000000000004000000000000000000000000000010000040000000000000000000000000000000000000000000000000000000100000000000ECFF93
:5C2E5C0000000000000480000000020000000001200000800010000240000000002000000000000000000008000100000000000000001000004000080000000000800010000200000000010000048000100002400008000020000400000028FF64
:5C2EB8000600000000000000000000000000000000000000000000000000000000000000000000000000000000000000000000000000000000000000000000000000000000000000000040000000000000000000000000000000000000C012FFA7
:5C2F1400000000808000080000000000000000000080000000000000000000000000000000000000000000000000000000000000000000000000000000000000000000000000000000000020000000000000000000200000000000000000F4FDA8
:5C2F700000000000000000010004000000000000000000000000000002000000000000000000000000000000080000000000000000000000000800080000000000000000000200000000800000200000000000000000000000000000000070FED6
:5C2FCC00000000000000000000000000000000000000000000000000000000000000000000000000000000000000000000000000000000000000000000000000000000000000000000000000000000000000000000000000000000000000DCFFCE
:5C302800000000000000000000000000000000000000000000000000000000000000000000000000000000000000000000000000000000000000000000000000000000000000000000000000000000000000000000000000000000000000DCFF71
:5C308400000000000000000000000000000000000000000000000000000000000000000000000000000000000000000000000000000000000000000000000000000000000000000000000000000000000000000000000000000000000000DCFF15
:5C30E000000000000000000000000000000000000000000000000000000000000000000000000000000000000000000000000000000000000000000000000000000000000000000000000000000000000000000000000000000000000000DCFFB9
:5C313C00000040000000000000000000000000000000000001000000000000000000000000000000000040000000000000000000000002002000400000000000000000000000000000000E0000000000000000000000000000000000000040FF07
:5C319800000000004000000000000000000000000000000000000000000000000000000000000000000000000000000000000000000000000000000000000000000000000000000000000022000000000000000000000000000000000000F8FD84
:5C31F40000000010000A4001000000000000000040000040000000000000000000000000000000000000001000000000000000000000280000A0000000000000000000280004000000000050000A00010000000000000000400008000008C0FC39
:5C3250000000000000000000400000000000000000001000020000000000000000000000000000000000000000000000000000000000000000000000000000000000000000000000A000000000000002400000000000000000000000000004FFEB
:5C32AC002000000000C0080240000000000000000000000000000000020000080000000004000000000000200000000000000000000000000002000000000086000000000000000000000000000000000000000001000000002000000200CCFFF8
:5C33080000000000000000010000000000000000000000000000000080000000020000000001000000000000000000000000000000000000008000000000000000000000000000000000000000000000000000000000000000000800000044FD1C
:5C3364006080000000F00006C8000100000000000000000000000018000060000000003000000000000000600000000000000000000000001800000000008007000000000000000000000000000000000000000003000000800100000600F0FD50
:5C33C000A011000000D0841A4123000000000000000000000000000800002000000000100000000000000020000000000000000000000000080000000000800608000000000000000000000000000000000000000100000080000000020030FF8E
:5C341C000004000000C042800410000000000000000000000000006004008009010000C02800000000000080090200000000000000000000600100000000000604000000000000000000000000000000000000000C0100000006020098006CFCD9
:5C347800C041000000E0001C808300000000000000000000000000708000C001000000E000000000000000C0010000000000000000000000701000000000000700000000000000000000000000000000000000000E000000000700001C04B8FF33
:5C34D4008041000000C000180803020000000000000000000000006000008001000000C00000000000000080010000000000000000000000600000000000000602000000000000000000000000000000000000000C00000000060000180094FFAF
:5C3530008001000000C022980003000000000000000000000000006000008001000000C00000000000000080010000000000000000000000600000000000004600000000000000000000000000000000000000000C0000000006000018007CFDD6
:5C358C000400000000C008020000000000000000000000000000000002000008000020000000400000000000080001000000000000000000080000000000008600000000100800000000000000000000400000000000000400200000800014FD07
:5C35E80000800000000000010000010000000000000000000000000080000000020000080000000000000000000240000000000000000000000000000000000000000000000400000000000000000000000000000000800000000800002074FF1A
:5C3644006800000000F00006C000000000000000000000000000001800006000008001000000C00001000060000C000000000000000000001800000000008007000000C0001800000000000000000000C00000000060000C800100000600D8FEE6
:5C36A0002000000000D0440240000000000000000000000000000008000020000080000000004023000000200004000000000000000000000800000000008086000000400008000000000000000000004000000000200004800000000280A8FEC7
:5C36FC008401000000C00818012301000000000000000000000000600100800900004601000000080000008045300A0000000000000000006000000000000016020000008B60140000000000000000000013000000801130210600001880ADFDFC
:5C375800C001020000E0801C880300000000000000000000000000701000C0410000070000008083000000C00138000000000000000000007080000000000007000000800370000000000000000000008083000000C00139000704001C04E8FECF
:5C37B4008801000000C0201800030000000000000000000000000060000080010000060000000083000000800130000000000000000000006000000000000006000000000360000000000000000000000003000000800130000600001800ADFCD6
:5C3810008001000000C002180003000000000000000000000000006000008001000006000000002300000080013000000000000000000000600000000000001604000000036000000000000000000000000300000080013000060000180038FC60
:5C386C00802104000000040200230000000000000000100000000008000000080000201000000023000000200004000000000000000000000800000000008000000000001008000000000000000000004000000000000000002000000200E4FFB6
:5C38C800000000000000000100000400000000000000000000000000000000000200000800000000040000000000000000000000000000000000000000000000000000000004000000000000000000000000000000008000100008000000CCFC2D
:5C392400E0010C0000300006C003000000000000000030000000001800006000008001300000C00300000060000C000000000000000000001800000000008001080000C0001800000000000000000000C00000000060000C80010000060024FE8B
:5C398000A84104000010000240230400000000000000100000000008000020000080001000004043000000200004000000000000000000000800000000008016000000400008000000000000000000004000000000200004800000000200EDFF5E
:5C39DC008041B00000C0201801230000000000000000C0200000006012008045000016C12000000B0000008005B008000000000000000000600400000000001000000000936084000000000000000000000B00000080113002160000180360FF63
:5C3A3800C001382000E0001C84830000000000000000E000000000700000C001000007E000008003020000C08138000000000000000000007020000000000007020000800370000000000000000000008003040000C08138080702001C0080FDEA
:5C3A94008441300000C0001800830000000000000000C0000000006000008001000006C000000003000000800130000000000000000000006000000000000006000000000360000000000000000000000003000000800130000600001880D8FE7A
:5C3AF0008011300000C00018000B0000000000000000C0000000006000008001000006C0000000A300000080013000000000000000000000600000000000004601000000036000000000000000000000000300000080013000060000180014FC2F
:5C3B4C0024000400001000000023000000000000002010000000106008002000000020100000001000000000080001000000000000020000000200000000800000000040000002002000000000000000400000000000003002460000020060FCB5
:5C3BA8000000000000000000080004000000000000000800000000040000000000000008000000000400000000024000000000000000000000800000000000000000000000008000000000000000000000000000000080004000080000007CFF18
:5C3C040068800C0000300006C0030000000000008001300000C0007810006000008001300000C00000000060000C000000000000000600001800000000008001080000C0001800006000000000000000C00000000060003C88070400060014FC5D
:5C3C6000A011040000100002400B020000000000800010000040006802002000008000100000400000000020000400000000000000020000080000000000801600000040000800002000000000000000400000000020003480160000028008FDED
:5C3CBC000404B10000C0201801230000000000000016C48800000B6000008089000006C1020000830000008005B008000000000000180800600400000000000000000000936001008005010000000000000B0000008009B200460000588085FC95
:5C3D1800C001384000E0001C88030100000000000007E000008003721000C001000007E020008003000000C04138000000000000001C000070100000000000070100008003701000C0010000000000008083000000C00138080701001C0498FFF3
:5C3D74008801300000C0001800830000000000000006C0000000036010008001000006C00000000300000080013000000000000000180000600000000000000601000000036000008001000000000000000300000080013008060000180021FD50
:5C3DD0008049300000C0001800230000000000000006C0000000036000008001000006C0000000030000008001300000000000000018000060000000000000060000000003600000800100000000000000030000008001B000160100180094FC2A
:5C3E2C0004000001001000180100000000000000000000040000100800008011008000000400400000000000080001000000000000020000080000000000800000000040000800008011000000000000001000000000000480000000800048FDD6
:5C3E8800008000400000000020000100000000000000000001000004000000000200000000010000000000000002400000000000000000000000000000000000000000000000000000000200000000000000040000008000000000000020B8FF56
:5C3EE40068000C000030401EC8000000000000000000300000C000180000E001008001300000C00000000060000C000000000000000600001820000000008001080000C000180000E041000000000000C00000000060000C80010200060054FF2A
:5C3F40002000040000D0085A400000000000000000001000004000080000A04100800010000040000000002000040000000000000002000068040000000080160000004000080000A0090000000000004000000000200004804600000280ACFD18
:5C3F9C008405B00000000818000B0000000000000000C02000000B6220008001000006C1200000200200008001B000000000000000980000008200000000002000000000A360010080090200000000000023000000809130022000005880F1FD28
:5C3FF800C001390800E0201CA0030100000000000000E000008003700000C041000007E000008000000000C04138080000000000001C040070000000000000070200008003701000C0010000000000008083000000C00138080701001C0428FD81
:5C4054008801300000C0801800030000000000000000C0000000036000008001020006C00000000301000080013000000000000000180000600000000000000600000000036000008041000000000000000300000080013000060400180059FF0B
:5C40B0008001300000C0081805030000000000000000C0000000036000008009000006C00000002300000080013000000000000000180000600800000000001601000000036000008001000000000000000300000080013000460000180014FF35
:5C410C0024000400000004020000000000000004000000048000100800002000048000000400400000000020000400000000000000800000600400000000800000000040006004002000000000000000001000000080110000460000808038FF37
:5C41680000000000000000010000010000000000000000000120000400000000000000000001000000000000000000000000000000002000008000000000000000000000000080000000000000000000000004000000000210000800002000FE77
:5C41C40068000C0000300006C80000000000000C0000300006C00018000060000C8001300000C00001000060000C000000000000000600007810000000008001000000C0007800006000000000000000C000000000E0010C800701000600F1FEF8
:5C422000200004000010001A41000000000000040000100002400008000020000480001000004023000000200004000000000000000200006800000000008000000000400068420020000000000000004000000000A0410480060000020068FF12
:5C427C000408B00000C0040005130400000000304200C0021801436001008009300216C8020000000000008011300A0000000000009804006000000000000010040000000B60020080090000000000000013000000804130010600009880CCFFFF
:5C42D80040003A0800E0401C80030000000000380000E0201C9003701000C001391007E020008003020000C00139000000000000001C000070100000000000010000008003721000C0010200000000008083000000C00138400701001C04BCFECF
:5C4334008881300000C0001800030000000000300000C0001800036000008001300006C0000000030000008001300000000000000018000060000000000000060800000003601000800100000000000000030000008041300006000018005DFE9C
:5C4390008011300000C0009804030000000000300000C0001800036000008001300006C00000008300000080013000000000000000180000601400000000001600000000036002008001000000000000000300000080113000160800180060FCBD
:5C43EC00240004000010001841000000000000000000000400002300020020000080001000004000000200801104000000000000008000000002000000008000000000400008000000000000000000000010000000801100002000001801A4FF6D
:5C44480000000000000000002000000000000000000000000100000480000000000000000000000000800000000200000000000000002000008000000000000000000000000000000080000000000000000004000000000210000800002098FDFE
:5C44A40068800C000030401EC0000000000000000000300000C0831800006000008001300000C000180000E0010C000000000000000600001800000000008001080000C0001800006000000000000000C000000000E0010C800100001E0034FFBB
:5C450000A011040000D0081A50000000000000000000100000400B08000020000080001000004000080000A04104000000000000000200000800000000008016000000400008000020000000000000004000000000A01106800000001A8438FFD4
:5C455C00041030010000009800080000000000000000C0040000136012008045000016C148000083600C00804930000000000000009800006001000000000040000000008B6001008045000000000000000B0000008005B020C600001881F5FD6E
:5C45B800C0013A0800E0201CA0800000000000000000E020008083700000C001000007E000008003700000C00138400000000000001C040070400000000000070100008003702000C0010000000000008083000000C04138000700001C10D4FF33
:5C4614008841300000C0201804030100000000000000C0000000836000008001000006C000000003600000800131000000000000001800006000000000000006010000000360000080010000000000000003000000800130000600001800C5FC5C
:5C4670008005300000C0089800230000000000000000C0000000236000008001000006C00000000360000080113000000000000000180000600000000000001600000000036000008001000000000000000300000080513000060000180870FEFE
:5C46CC00000000810010000040000800012000000000100000400000020120000080001000804000000000801130020000000000000200000800000000008000000000001000020100000081000000004000000200000000800010000200C0FC64
:5C472800008000400000000008000000000000000000000000000000800000000000000000002000000000000002400000000000000000000000000000000000000000000004800000800040000000000000008000008000100000000000C0FD7A
:5C47840060000C8001300006C0001900036000000000300000C0001900036000008001300006C000000000E0013C000000000000000600001820000000008001080000C00018000360000C8001000000C00018000060000C800132000600B0FC42
:5C47E000280004800010000240230800012000000000100000402308000120000080001000024000000000A0213408000000000000020000680400000000801600000040000800012000048000000000400008000020000480461000020069FF2B
:5C483C008011310126C40418010060804C9085000000C00400001060228C8009000046C12818010B02000080053201000000000000980400001100000000004000000000A360144C800930212600000000236002008005300920C002190040FCD3
:5C489800C001380807E0401C840372000EC001000000E02000800372000ED041000007E0001C8803000000C00138100000000000001C00007000000000000007040000800370000EC8413800070200008083704000C081380007E4001C0430FFC5
:5C48F4008401300006C00018000360000C8001000000C00000000360000C8001000006C000180003000000800130000000000000001800006010000000000006010000000360000C800130000600000000036000008001300006C100188088FCF7
:5C4950008001300006C00018009360000C8001000000C00000002361000C8001000006C000180003000000805130200000000000001800006004000000000046000000000360000C800130000600000000036000008001300046C000180090FF80
:5C49AC00040000000000000000000000000000000000000000000000000000000000000000000000000000000000000000000000000000000000000000000000000000000000000000000000000000000000000000000000000000000000D8FFD4
:5C4A0800200004800010000240000800012000048000100002400008000120000480001000024000080001200004000000000010000240000800012000048000100002400008000120000480001000024000080001200004800010000200BCFC6A
:5C4A6400080000000000000000000000000000000000000000000000000000000000000000000000000000000000000000000000000000000000000000000000000000000000000000000000000000000000000000000000000000000000D4FF1B
:5C4AC00020000480001000024000080001200004800010000240000800012000048000100002400008000120000400000000001000024000080001200004800010000240000800012000048000100002400008000120000480001000028034FCBA
:5C4B1C0004012000048000100002400008000120000480001000024000080001200004800010000240000000012000000000000000100000400000000000000400000000024000080001200004000000000240000800012000048000108051FF91
:5C4B7800000000000000000000000000000000000000000000000000000000000000000000000000000001000000000000000010000040000000012000040000100002000000000000000000001000020000000000000000000000000000BCFE8D
:5C4BD4008800100002400008000120000480001000024000080001200004800010000240000800012000008000100000000000000008000020000000000000020000000001200004800010000200000000012000048000100002400008004DFEC9
:5C4C3000000000000000000000000000000000000000000000000000000000000000000000000000000001000000000000000010000040000000012000040000100002000000000000000000001000020000000000000000000000000000BCFED4
:5C4C8C00000000000000000000000000000000000000000000000000000000000000000000000000000000000000000000000000000000000000000000000000000000000000000000000000000000000000000000000000000000000000DCFFF1
:5C4CE800000000000000000000000000000000000000000000000000000000000000000000000000000000000000000000000000000000000000000000000000000000000000000000000000000000000000000000000000000000000000DCFF95
:5C4D4400000000000000000000000000000000000000000000000000000000000000000000000000000000000000000000000000000000000000000000000000000000000000000000000000000000000000000000000000000000000000DCFF38
:5C4DA000000000000000000000000000000000000000000000000000000000000000000000000000000000000000000000000000000000000000000000000000000000000000000000000000000000000000000000000000000000000000DCFFDC
:5C4DFC0000000100000000000000000000000000000000000000000000000040000000000000400000000000000000000000000000000000000000000000000000000000000000000000000000000000000000000000000000000000000088FF53
:5C4E580000000000000000000000000000000000000000000000000000000000000000000000000000000000080000000000000000000000000000000000000000000000000000000000000000000000000000000000000000000000000054FFA3
:5C4EB400000000000000000000000000000000000000000000000000000000000000000000000000000000000000000000000000000000000000000000000000000000000000000000000000000000000000000000000000000000000000DCFFC7
:5C4F1000000000000000000000000000000000000000000000000000000000000000000000000000000000000000000000000000000000000000000000000000000000000000000000000000000000000000000000000000000000000000DCFF6A
:5C4F6C00000000000000000000000000000000000000000000000000000000000000000000000000000000000000000000000000000000000000000000000000000000000000000000000000000000000000000000000000000000000000DCFF0E
:5C4FC800000000000000000000000000000000000000000000000000000000000000000000000000000000000000000000000000000000000000000000000000000000000000000000000000000000000000000000000000000000000000DCFFB2
:5C502400000000000000002000000000000000000020000000000000000000000000000000000000080000000000000000000000000000000000000000000000000000000000000000000000000000000000000000000000000000000000F4FFF5
:5C508000000000000000000000000000000000000000000000000000000000000000000000000000000000008000000000000000000000000000000000000000000000000000000000000000000000000000000000000000000000000000D4FF81
:5C50DC00000000000000000000000000000000000000000000000000000000000000000000000000000000000000000000000000000000000000000000000000000000000000000000000000000000000000000000000000000000000000DCFF9D
:5C513800000000000000000000000000000000000000000000000000000000000000000000000000000000000000000000000000000000000000000000000000000000000000000000000000000000000000000000000000000000000000DCFF40
:5C519400000000000000000000000000000000000000400000000000000402000000020100000000000000000000000000000000000000000000000000000000000000000000100000000000000000000000000000000000000000000000C8FCA2
:5C51F000000000000000000000000000000000000000000000000000000000000000000000000000000000000000000000000000000000000000000000000000000000000000000000000000000000000000000000000000000000000000DCFF88
:5C524C000000000000000000000000000000000000002000000000000002040000000102000000000000000000000000000000000000000000000000000000000000000000002000000000000000000000000000000000000000000000008CFE33
:5C52A800800000000040000000A0000000000000000000020000000000600000000A22410000000000000080020000000000000000000000000000000000000000000000A10016000000000000000000000000000020021000000000000084FC90
:5C530400800000000040000000800000000000000000000000000000000000000008024100000000000000800000000000000000000000000000000000000000000000008100100000000000000000000000000000000010000000000000A4FC01
:5C536000000000000000000000000000000000000000000000000000000000000000000000000000000000000000000000000000000000000000000000000000000000000000000000000000000000000000000000000000000000000000DCFF16
:5C53BC00000000000000000000000000000000000000000000000000000000000000000000000000000000000000000000000000000000000000000000000000000000000000000000000000000000000000000000000000000000000000DCFFBA
:5C541800000000000000000000000000000000000000000000000000000000000000000000000000000000000000000000000000000000000000000000000000000000000000000000000000000000000000000000000000000000000000DCFF5D
:5C547400000000000000100000000000000000000000000000000000000000000000000000000000000000000000000000000000000000000000000000000000000000000000000000000000000000000000000000000001000000000000DCFFF0
:5C54D000000000000000110000280000000000000000000000000000000000000000000000000000000000000000000000000000000000000004000000000000000000000000000000000000000000000000000000000000000000000000B4FE91
:5C552C00000000000000000000000000000000000000000000000000000000000000000000000000000000000000000000000000000000000000000000000000000000000000000000000000000000000000000000000000000000000000DCFF48
:5C558800000000000000000000000000000000000000000000000000000000000000000000000000000000000000000000000000000000000000000000000000000000000000000000000000000000000000000000000000000000000000DCFFEC
:5C55E400000000000000000000000000000000000000000000000000000000000000000000000000000000000000000000000000000000000000000000000000000000000000000000000000000000000000000000000000000000000000DCFF90
:5C564000000000000000000000000000000000000000000000000000000000000000000000000000000000000000000000000000000000000000000000000000000000000000000000000000000000000000000000000000000000000000DCFF33
:5C569C00000000000000000000000200000000000000000000000000000000000000000000000000000000000000000000000000000000000000000000000004000000000000000000000000000000000000000000000000002000000000BCFFD1
:5C56F8000000000000000000000000000000000000000000000000000000000000000000000000000000000000000000000000000000000000800000000000000000000000000000000000000000000000000000000080000000000000005CFFFB
:5C575400000000000000000000000000000000000000000000000000000000000000000000000000000000000000000000000000000000000000000000000000000000000000000000000000000000000000000000000000000000000000DCFF1E
:5C57B000000000000000000000000000000000000000000000000000000000000000000000000000000000000000000000000000000000000000000000000000000000000000000000000000000000000000000000000000000000000000DCFFC2
:5C580C00000000000000000000000000008000000000000000000000000000000000000000000000000000000000000000000000000000000000000000000000000000000000000000000000000000000000000000000000000000000000D4FFED
:5C58680000000000000000000000000000000000000000000000002000008000000000000000000000000000000000000000000000000000000000000000000000000000000000000000000000000000000000000000000000000000000054FDF3
:5C58C40000080000008000080000000000000000000000000000000000000010400000000020000000000000000004000000000000000000080000000000000000000000000000800008010000000000000000040000000021000000200298FD17
:5C59200000000200200000000040010000040000000000000040000000000008000000000000000000000000000040000000000000000000000000000000000000000000000008000080000100000000000000000000000001000000000058FD5D
:5C597C00000000000000000000000000000000000000000000000010000000000000000200000000000000000000000000000000000000000000000000000000000000000000000000000000040000000000000000000000000000000000D8FCE5
:5C59D80000000000000000000000000000000000080000000000000000000000000000000000000000000000000000000000000000000000000000000000000000000000000000000000000000000000000002000100000000000000000064FD07
:5C5A3400000000000000000000000000000000000000000000000000000000000000000000000000000000000000000000000000000000000000000000000000000000000000000000000000000000000000000000000000000000000000DCFF3B
:5C5A9000000000000000000000000000000000000000000000000000000000000000000000000000000000000000000000000000000000000000000000000000000000000000000000000000000000000000000000000000000000000000DCFFDF
:5C5AEC00000000000000000000000000000000000000000000003000000000000000000000000010000000000020000000000000000400000000000000000012080000000000000000000000000000000000000000000000000100400000C0FFE0
:5C5B48000014002000000000A000000000000000000000020000000000000000000000200000000000000000000000000000000000000000002000000000000000000000204000000000000000000000000000000000000000040000000020FC6B
:5C5BA400160000000000000000000000000000000000000000000000000000000000000000000000000000000000000000000000000000000000000000000000000000000000000000000000000000000000000000000000000000000000E8FDAA
:5C5C0000000000000000000000000000000000000000000000000000000000000000000000000000000000000000000000000000000000000000000000000000000000000000000000000000000000000000000000000000000000000000DCFF6D
:5C5C5C008040000002408000008100000020000000004020000081000000024000000001000000000000000040000000000000000008100000000020000000000000000000001000404000000000000400810000042000000000402008008CFF01
:5C5CB80000000000000000000000000000000000000000000000000000000000000000000008000000000000000000000000000000004000000000000000000000000000000000010000000000000000000000000000000000000000000090FEB9
:5C5D14004080000001204000800001000440000000002040008000010000048000000002000A000000000000800000000000000000044800000000400000000000000000000020014080000000000004800001000240000000002040040010FFB5
:5C5D7000803E000810000200441000002420000020400100240010000044805000262240214811002000808208100A000000000000088404000000000044000000000000A1000004004010000400000000812000A00100100E02000648046CFE8D
:5C5DCC0080000020000000001000000004000000000001000000000000048040008000402008000040000082001008000000000000080400000000000000000000000000810000040020100000000000008120000000001008020000080444FD77
:5C5E280000400000000000000000000000000000000000000000000000000000000800000000000000000000000000000000000000000000000000000000000000000000000000000000000002000000000000000002000010000000000048FF7B
:5C5E840000000020000080000000000000000000000004800010000240000000010000048000100002400000000120000000000000001000004000000000000000000000000240000000002000000000000002400000000000000400001088FDC7
:5C5EE0001A020000000000200004000000000000000000000000000000000000000000000000000000000000000000000000000000000000000000000000000000000000000000000002000000000000000000000000024000000000000086FF5D
:5C5F3C0000000200000000041200000000000000000000000000020000000000000000000000000000000000000000000000000000000000000000000000008000000000000000000000000000000000000000000000000080000000020090FE5F
:5C5F980000000000000004000002000000000000000000000000000000000000000000000000002800000000010000000000000000000000000000000000000000000000000010000000000000000000000000000000000000A00000000040FC92
:5C5FF400000000000000000000000000000000000000000000000000000000000000000000000000000000000000000000000000000000000000000000000000000000000000000000000000000000000000000000002000000000000000FCFD38
:5C6050000000000000000000000000000000000000000000000000000000000000000000000000000000000000000000000000000000000000000000000000000000000000000000000000000000000000000000004000000000000000009CFF19
:5C60AC00000000000000000000000000000000000000000000000000000000000000000000000000000000000000000000000000000000000000000000000000000000000000000000000000000000000000000000000000000000000000DCFFBD
:5C61080000000000000000000000000000000000000000000000000000000000000000000000004000000000000000000000000000000000000000000000000000000000000000000000000000000000000000000000000000000000000098FF64
:5C61640000000000004000000004000000000000000000000002000080001000000000000000000000000020A00000000000000000000000800000000000802000000000000000000000000000000000000000000000020000400000000030FEB9
:5C61C000000000020000000000000000000000000000000000002000000000000000000000000000000000000000000000000000000000000000000000000046000000000000000000000000000000000000000000000000000004000000B8FF60
:5C621C0000000000000000012000041000000000000000000000000400000000020000000000000004000000000240000000000000000000008000000000000002000000000080000000020000000000000000000000000240000800002074FDC6
:5C627800A0000000004000080001000000000000000000000000010800000000000000000000000100000000000000000000000000000000200000000000800000000000000000000000000000000000000000000000010000020000000018FE1E
:5C62D4000000040000000000001008000C0100000000000480001000000000000000000000800000000000000000000000000000000200000002000000000000000000000000020000000000001000800000000000000000000000040000C0FED9
:5C633000000000000000000000000400000000000000000001200004000000000000000000002000000000000000000000000000000000000080000000000000000000000000800000000000000000002000000000000000000000000100E0FEC9
:5C638C0000000C4000000000C00018800F0000000000300006C0000000000000000000000006000000000000000000000000000000060000180000000000000000000000001800000000000000300006000000000000000000003000000040FF2B
:5C63E8000000B40000000000400068012D0200000000100002400000000000000000000000020000000000000000000000000000000200000800000000000000000000000008000000000000001000020000000000000000000010000000B8FF8E
:5C6444000000000100000000008B00024C0000000000C002580043000000000000000000001810000000000000000000000000000098080060110000000000000000000000600C000000000000C0021801000000000000000000C022000084FFE0
:5C64A0000000380800000000800370100E1000000000E0201C8403000000000000000000001C0000000000000000000000000000001C0000700000000000000000000000007000000000000000E0401C04000000000000000000E00000002CFF39
:5C64FC000000300000000000000360800C0800000000C0001800030000000000000000000018000000000000000000000000000000180000600000000000000000000000006000000000000000C0001800000000000000000000C0000000BCFE00
:5C6558000000301100000000000360042C0000000000C0001800030000000000000000000018000000000000000000000000000000180000600000000000000000000000006000000000000000C0001800000000000000000000C0000000DCFFD5
:5C65B4000000000100000000400000000100000000200004800010000000000000000000008000000000000000000000000000000002000000000000000000000000000000000200A010000000000402000000000000000080000004000098FC43
:5C66100000000040000000000000002000000000000008000120000400000000000000000000200000000000000000000000000000000000000000000000000000000000000080000001020000000001000000000000000000000000010044FCBC
:5C666C0000000C0000000000C0001800030000008001300006C000000000000000000000000600000000000000000000000000000006000000000000000000000000000000180000E000000000300006000000000000000080013000000048FD44
:5C66C800040004000000000040000800010000008000100002400000000000000000000000020000000000000000000000000000000200000000000000000000000000000008000020010000001000020000000000000000800010000080B4FF51
:5C6724000C00301000000000009360112C0200000026C02898000B0000000000000000000058000000000000000000000000000000580000000000000000000000000000006004008000000000C0241802000000000000000046C12000808DFC28
:5C6780000000380000000000800370000E0000000007E1001C9003010000000000000000001C0400000000000000000000000000001C0400000000000000000000000000007040004001000000E0001C00000000000000000007E000000010FDCB
:5C67DC000800300000000000000360000C0000000006C0001800030000000000000000000018000000000000000000000000000000180000000000000000000000000000006000008000000000C0001800000000000000000006C00000002DFFFF
:5C6838000000300000000000000360000C0000000006C0001800030000000000000000000018000000000000000000000000000000180000000000000000000000000000006000000001000000C0001800000000000000000006C0000000ACFFAA
:5C6894000400000120000000001000000000000080001000020010000000000004000000000200000000000008000000000000C01002000000000000000000000000000000600800200000000010008000100002400000008000C010020024FD14
:5C68F00000000040000800000000042000040000000000000000000400000000000000000000000000000000000200000000000000000000000000000000000000000000000000000000000000000000200004800010000000000000000040FFE3
:5C694C0008000C8001000000C0001800030000008001300006C00000000000000C000000000600000000006000000000000000F020060000000000000000000000000000007800006000000000300006C0001800030000008001F0400600A0FF41
:5C69A8000000048000000000400008000100000080001000024000000000000004000000000200000000002000000000000000D00202000000000000000000000000000000681200200000000010000240000800010000008000D004028008FF28
:5C6A04000400B02006000000002360148C02000000C6C004980013040000000030010000009800000000008009000000000000C084980000000000000000000000000000006002008011000000C00058104360028C0800000046C0001891B5FD1B
:5C6A60000000380007080000808370000E0000000007E0201C9003000000000038080000001C1000000000C041000000000000E0001C040000000000000000000000000000704000C041000000E0201C800370100E0000000007E1201C008CFE63
:5C6ABC000800300006000000000360000C0000000006C000180003000000000030000000001800000000008001000000000000C020180000000000000000000000000000006000008001000000C00018000360000C0000000006C00019002DFEFD
:5C6B18000000300006000000000360000C0000000006C000180003000000000030000000001800000000008001000000000000C000180000000000000000000000000000006024008001000000C00018000360000C0000000006C008180038FE92
:5C6B7400240030048600000200436008000000008000100018420000000000000400000000180200000000200000000000000000000200000002000000008000000000000060080020000000000004180110080001000000002010000000E4FDBF
:5C6BD000000000000000000000000000000400000000000000000000000000000000000000000000000000000000000000000000000000000080000000000000000000000000000000000000000000012000040000000000000008000000A4FC18
:5C6C2C0068003C8007000006C003780003000000800130001EC80004000000000C000000001E00000000006000000000000000000006000018000000000080010000000000780000600000000030001EC000180003000000800130000100B8FD71
:5C6C88002000B488260400024093681001000000800010001A400B000000000004000000009A04000000002000000000000000000002000008000000000080000000000000681000200000000010005A44000800010000008000D0020080A8FDD5
:5C6CE4008405300116000098042362022C0200000016C1021800900000000000302200000018010000000080010200000000000000180000601400000000000602000000006010008005000000C00218009360084C0000000046010200804DFF05
:5C6D4000C0013A100701001C800370800E0000000007E0401C8403000000000038000000001C0400000000C00100000000000000001C040070000000000000070000000000700000C041000000E0201C840370000E0800000007E020000080FCB0
:5C6D9C008801304006010018000360800C0000000006C0001800030000000000300000000018100000000080010000000000000000180000600000000000000600000000006000008001000000C00018040360000C0000000006C000000089FDE4
:5C6DF8008001300146000018008B60000C0000000006C0005808130200000000300000000018000000000080010000000000000000180000600000000000000600000000006021008001000000C00098000360000C0000000006C04200002CFEBB
:5C6E5400000804002000000240006008000000000020C010180223000000000000010000000200000000002000000000000000100080000000000000000000000000800000080000200000000010000240000002400000000020C010008090FEF2
:5C6EB0000000020000080000000000000004000000000800000000040000000000400000000000000000000000000000000000000000200000000000000000000000002000000000000000000000000000000080001000000000080000008CFDCB
:5C6F0C0060000CC001000006C0007800030000008001F0001EC00300000000000C0000000006200000000060000000000000003000060000000000000000000000000600001820006000000000300006C0001800030000008001F000000075FE0E
:5C6F68002800B4800000000240006811010000008000D0205A5083000000000004000000005A00000000002000000000000000100002000000000000000000000000020000680400200000000010000240000800010000008000D08000000CFFC4
:5C6FC4008009800816010018040361414C0000000016C0801801A30000000000B0000000008000000000008051000000000000C018180100000000000000000000001808000081008009000000C00000211360022C0200000046C0080080BCFD43
:5C702000C04138000700001C800370000E0800000007E1001C8403000000000038080000001C0800000000C001000000000000E0001C0400000000000000000000001C0000700000C041000000E08004800371400E0000000007E12000006CFE5A
:5C707C008401300006000018000360000C0000000006C000180003020000000030000000001804000000008001000000000000C000180000000000000000000000001800006010008001000000C00018200360000C0000000006C000000055FD66
:5C70D8008001300906000018000360440C0000000006C02418020B000000000030000000005800000000008001000000000000C000180000000000000000000000001800006001008001000000C00058000360000C0000000006C084000050FEC8
:5C71340004083084000000804000080001000000800000040200230800000008000100000002000000000020000400000000000004800000080000000000000000000000000800002000000000000402001060040100000080001000000044FE95
:5C719000000002000000000020000000000000000000000001000004000000000240000000000000000000000000000000000000000120000000000000000000000000000000000000000000000000010000048000000000000000000000F4FDA3
:5C71EC0068003C8001000006C0001800030000008001300006C00318000060000C0000000006000000000060000C00000000003000060000180000000000000000000000001800006000000000300006E00078000300000080013000000038FD94
:5C7248002000348800000002400008000100000080001000024093080000200004000000000200000000002000040000000000100002000008000000000000000000000000080000200000000010005A400068110100000080001000000091FF86
:5C72A4008441300A26000018041362018C0200000016C00440200B608100801131010000000001000000008009301200000000C024180000608200000000000000000000000001008049000000C00080002362028C1000000016C08000009CFE99
:5C730000C00138000704001C800370200E0000000007E120048083700000C0013808000000041000000000C041380000000000E0001C040070000000000000000000000000101000C001000000E0201C840370200E0000000007E1000000B0FEFB
:5C735C008801302006000018000360000C0000000006C000180403600000800130000000001820000000008001300000000000C000180000600000000000000000000000006020008001000000C00018040360100C0000000006C00000809CFE1C
:5C73B8008001300206000018000360000C0000000006C000180143600000800130000000005800000000008001300000000000C000180000600000000000000000000000006004008001000000C00018010360040C0000000006C000000058FF77
:5C74140024000081000000800010080001000000002010000200100000000000040000100002000008000120000000000000000004800000080000000004000000000000000800002000000000C01002002308000C01000080001000008048FC47
:5C74700000000040000000002000040000000000000008000000000400000000000000000000000000000000000000000000000000012000000000000000000000000000000000000000000000000000000004000000000000000000000094FE99
:5C74CC0068000C8001080006C0001800030000008001300006E00000000000000C000030000600001800036000000000000000300006000018000000000C000000000000001820006000000000F00006C08318000F0000008001300001008DFFA2
:5C75280020000480160000024000080001000000800010005A40000000000000040000100002000008000120000000000000001000020000080000000004000000000000006804002000000000D02802400B08002D0200008000D002000094FC91
:5C7584008441301120000098009360114C1000000016C1088000230200000000B00000C08058000060000C8811000000000000C0825800006011000000B0100000000000000002008041000000C00818010B60024C0200000016042400808CFC4C
:5C75E000C00138000701001C840370000E0000000007E0401C84030000000000380800E0001C040070400EC081000000000000E0001C040070000000003800000000000000701000C001000000E0201C848370100E0000000007E00000002CFD7A
:5C763C008801300006000018000360000C0000000006C0001804030000000000300000C00018000060000C8001000000000000C000180000600000000030000000000000006010008001000000C02018000360000C0200000006C000000001FC4D
:5C7698008001300006040018000360000C0000000006C0005800030000000000300000C00018000060000C8001000000000000C000180000600000000030000000000000006004008001000000C0041800A360004C0000000006C028000088FF51
:5C76F4002400048000100002400008000C01000081001000024000000001000000810000000200100000000008000000000000100002001008000020000000000004000000000200200000000000048040000800402000000020100000806CFC08
:5C775000000000000000000000000000000000004000000000000000000000000040000000000000040000000002000000000000000000000400000000000000000001000000800000000000000000012000000000100000000008000000CCFCD1
:5C77AC0068000CC001000006C0001C800F00000C8001300007C00004000300000C8001000006E0000000006000000000000000300006C000180000600000000030000000001800006000000000300006C000188003600000800130000000B5FF11
:5C7808002000B48000000002400B68018D0200048000D00202400B000001000004800000005A4000000000200000000000000010000240000800002000000000100000000008000020000000001000024000680101200000800010000000DCFEB1
:5C7864008409800016C10818001000124C0200B00026002458008800002C0800300A4608008000230400008051000000000000C02418010B6014008011000000C0820000006040008045000000C04098009300114C8009000016C02200802CFFDE
:5C78C000C041384007F0001DA08370000E0000381007E1001C840300000E000038000700001C8403000000C001000000000000E0001C8403710000C001010000E000000000700000C001000000E0001C900370000EC201020007E1000000D8FC65
:5C791C008801300006C00018000360000C0800300006C00019000301000C000030000600001804030000008001000000000000C0001800036000008001000000C0000000006000008001000000C00018000360400C8001000006C00000002DFCB8
:5C7978008001300406C00018000B62124C0000300006C00418000B00000C000030000600001801030000008001000000000000C0001800036000008001000000C0000000006000008001000000C00018000360040C8001000006C000000018FF53
:5C79D400040000000000000000000000000000000000000000000000000000000000000000000000000000000000000000000000000000000000000000000000000000000000000000000000000000000000000000000000000000000000D8FF7C
:5C7A3000200004800010000240000800012000048000100002400008000120000480001000024000080001200004000000000010000240000800012000048000100002400008000120000480001000024000080001200004800010000200BCFC12
:5C7A8C00080000000000000000000000000000000000000000000000000000000000000000000000000000000000000000000000000000000000000000000000000000000000000000000000000000000000000000000000000000000000D4FFC3
:5C7AE80020000480001000024000080001200004800010000240000800012000048000100002400008000120000400000000001000024000080001200004800010000240000800012000048000100002400008000120000480001000028034FC62
:5C7B4400040120000400001000024000080000200004800010000240000800012000048000100002400008000120000000000080001000024000000001200004800010000040000000010000008000100002400008000100000480001080E5FEAA
:5C7BA00000000000001000000000000000200000000000000000000000000000000000000000000000000000000000000000000000000000000001000000000000000040000000010000048000000000000000000000000400000000000020FC73
:5C7BFC00880010000200000800012000040000100002400008000120000480001000024000080001200004800010000000000040000800012000008000100002400008000020000080000000004000080001200004800000000240000800B5FC8D
:5C7C580000000000001000000000000000200000000000000000000000000000000000000000000000000000000000000000000000000000000001000000000000000040000000010000048000000000000000000000000400000000000020FCBA
:5C7CB400000000000000000000000000000000000000000000000000000000000000000000000000000000000000000000000000000000000000000000000000000000000000000000000000000000000000000000000000000000000000DCFF99
:5C7D1000000000000000000000000000000000000000000000000000000000000000000000000000000000000000000000000000000000000000000000000000000000000000000000000000000000000000000000000000000000000000DCFF3C
:5C7D6C00000000000000000000000000000000000000000000000000000000000000000000000000000000000000000000000000000000000000000000000000000000000000000000000000000000000000000000000000000000000000DCFFE0
:5C7DC800000000000000000000000000000000000000000000000000000000000000000000000000000000000000000000000000000000000000000000000000000000000000000000000000000000000000000000000000000000000000DCFF84
:5C7E2400000000000000000000000000000000000000000000000000000000000000000000000000000000000000000000000000040000000000000000000000000000000000000000000000000000000000000000000000000000000000D8FF27
:5C7E8000000000000000000000000020000000000000000000000000000000000000000000000000000000000000000000000000000000000000000000000000000000000000000000000000000000000000000000000000000000000000DCFDAD
:5C7EDC00000000000000000000000000200000008000000000000000000000000000000000000000000000000000000000000000000000000000000000000000000000000000000000000000000000000000000000000000000000000000F4FFB7
:5C7F3800000000000000000000000000000000000000000000000000000000000000000000000000000000000000000000000000000000000000000000000000000000000000000000000000000000000000000000000000000000000000DCFF12
:5C7F9400000000000000000000000000000000000000000000000000000000000000000000000000000000000000000000000000000000000000000000000000000000000000000000000000000000000000000000000000000000000000DCFFB6
:5C7FF000000000000000000000000000000000000000000000000000000000000000000000000000000000000000000000000000000000000000000000000000000000000000000000000000000000000000000000000000000000000000DCFF5A
:5C804C00000000000000000000000000000000000000000000000000000000000000000000000000000000000000000000000000000000000000000000000000000000000000240000000000002000000000000000000000000000000000D8FDBF
:5C80A800000000000000000000000000000000000000000000000000000000000000000000000000000000000000000000000000040000000000000000000000000000000000000000000000000000000000000000000000000000000000D8FFA1
:5C810400000000000000000000000000000000000000000000000000000000000000000000000000000000000000000000000000000000000000000000000000000000000000000000000000000000000000000000000000000000000000DCFF44
:5C816000000000000000000000000000000000000000000000000000000000000000000000000000000000000000000000000000000000000000000000000000000000000000000000000000000000000000000000000000000000000000DCFFE8
:5C81BC00000000000000000000000010000000000000002000000000000000000000000000000000000000000000000000000040000000000010000000000000000000000000000000000000000000000000000000000000000000000000B8FD32
:5C82180000000000000000000000000000000000000000000000000000000000000000000000000000000000000000000000000000000000400000000000000000000000000000000000000000000000000000000000000000000000080050FF73
:5C82740000000000000000000000002000000000000000400000000000000000000000000000000000000000000000000000002000000000082000000000000000000000000000000000000000000000000000000000000000000000020050FFB5
:5C82D0000000000000000000000000160000000000000004000001000000000000000000000000000000000000000A00000000000008000020000000000000020000000000000000000000008000200000000000000000000004000000009CFDC6
:5C832C00000000000000000000000010000000000000000000000100000000000000000000000000000000000000080000000000000800002000000000000002000000000000000000000000000080000000000000000000000000000000D4FD61
:5C83880000000000000000000000000000000000000000000000000000000000000000000000000000000000000000000000000000000000000000000000000000000000000000000000000000040000000000000000000000020000000098FDFE
:5C83E400000000000000000000000000000000000000000000000000000000000000000000000000000000000000000000000000000000000000000000000000000000000000000000000000000000000000000000000000000000000000DCFF62
:5C844000000001000000000000000000000000000000000000000000000000000000000000000000000000000000000000000000000000000000000000000000000000000000000000000000000000000000000000000000000000000000CCFF14
:5C849C0000000000000000000000000000080000000000000000000000000000000000000000000000000000000000000000000000000000000000000000000000000000000000000000000000000000000000000000000000000000000054FF29
:5C84F800000000000000000000000000000000000000000000000000000000000000000000000000000000000000000000000000000000000020000000000000000000000000000000000000000000000000000000000000000000000000DCFD2F
:5C8554000000000000000000000000000000000000000000000000000000000000000000000000000000000002000000000000000000000000000000000000000000000000000000000000000000008000000000000000000000000000005CFDF0
:5C85B000000000000000000000000000000000000000000000000000000000000000000000000000000000000000000000000000000000000000000000000000000000000000000000000000000000000000000000000000000000000000DCFF94
:5C860C00000000000000000000000000000000000000000000000000000000000000000000000000000000000000000000000000000000000000000000000000000000000000000000000000000000000000000000000000000000000000DCFF37
:5C866800000000000000000000000000000000000000000000000000000000000000000000000000000000000000000000000000000000000000000000000000000000000000000000000000000000000000000000000000000000000000DCFFDB
:5C86C400000000000000000000000000000000000000000000001000000000000000000002400200000000000000000000000000000000000000000000000000000000000000000000000000000000000000000000000000000000000000ACFC5E
:5C872000000000000000000000000000000000000000000000000000000000000000000000000000000000000000000000000000000000000000000000000000000000000000000000000000000000000000000000000000000000000000DCFF22
:5C877C00000000000000000000000000000000000000000000000000000000000000000000000000000000000000000000000000000000000000000000000000000000000000000000000000000000000000000000000000000000000000DCFFC6
:5C87D800000000000000000000000000000000000000000000000000000000000000000000000000000000000000000000000000000000000000000000000000000000000000000000000000000000000000000000000000000000000000DCFF6A
:5C8834000000000000000000000000000000000000000000000000000000000000000000000000000000200000000000000000000000000000000000000000000000000000000000000000000000000000004000000000000000000000009CFDEF
:5C88900000000000000000000000000000000000000000000000000000000000000000000000000000000000000000000000000000080000000000000000000000000000000000000000000000000000000000020000000000000000000054FD31
:5C88EC00000008010000000000000000000000000000000200010100004000000000000000100000000000000000000000000010000000000000000020000001000404000008090000000000000000000000000000000000002000020000C4FEA5
:5C89480000000000800000000010001000000000000000000000000000000000000000000000000000000000000000000000000000000002000000000000000000000000000000000000000000801000000800000000000000000000400068FDF4
:5C89A40000000000400000010000000000000000000000000040000020000000000000000000000000000000000000000000000000000000000000000010000000000000000000000000020000000000010200000000000100000000000098FD2B
:5C8A000000000000000000000000000000040000000000000000000000000000000000010000000000000000000800000000000000000000000000000000000000000000000000000000000000000000000000000000000000000000000018FEF7
:5C8A5C00000000000000000000000000000000000000000000000000000000000000000000000000000000000000000000000000000000000000000000000000000000000000000000000000000000000000000000000000000000000000DCFFE3
:5C8AB800000000000000000000000000000000000000000000000000000000000000000000000000000000000000000000000000000000000000000000000000000000000000000000000000000000000000000000000000000000000000DCFF87
:5C8B140000000000000000008000004600000000000000210000000000000000000000000000000000000000000000000000000000000000000000000000000000000000000000000000000000000000000000000000000000002000000050FEB0
:5C8B70000000000000000000002000000000002000008000000000010000000400000000000000000008000000000000000000000000000000000000000000000000000000000000000000000000000004000000000000000000800000000CFF4D
:5C8BCC000C0000000000000000000000000000000000000000000000000000000000000000000000000000004000000000000000000000000000000000000000000000000000000000000000000000000000000000000000000000000040B2FD12
:5C8C28000000002000080000200000000000000000000000000000000000000000000000000000000000000000000000000000000000000000000000000000000000000000000000000000000000000000000000000000000000000000007CFD2F
:5C8C840080400008024000080481000004000000000241000000010000000000000800000008000000000000000000000000004020000000200000000000000000200000002000000000000000000000000100000000000080000000000044FE22
:5C8CE00000000000000000000000000000000000000000000000000000000000000002000000000020000000000000000000000000004000000000000000000000000800000000040000000000400008000000000000000000004100000004FD40
:5C8D3C004080001001200004880001000200000000012200008000000000000000900000000400000800280000000000000000204000400010000000000000000040020000100029000000000010000280000000000000000001140000009CFC8A
:5C8D9800204200000010022200100000A4820200000010220000AA004004004010081200000800020000008040502000000000402E080000200100810010004004044000000000200000000000002000020A08140020106104024100080010FDE8
:5C8DF40000400000000000000000000004820000000000200000800000040040100802000008000000000080401000000000004020080000200000800020000000000000000000000000000000002000000000100000000000014100040020FDCC
:5C8E500000000000000000000000000000000000000000000000010000000000000000000000000100000000000000000000000000000000000000010000000000000000000000000000000000000000040100000000001010000000000088FE18
:5C8EAC0000000120000400001000020000000000200004800010000200000000012000000000100002000000000100000000000080001000024000000000000000800010000040000000000000008000100002400008000000000480000078FED3
:5C8F08001E000000000000000000800010000000000000000000000000000000000000000000000000000000000000000000000000000000000000000000000000000000000000000000000000000000000000000000000000000000008061FC82
:5C8F640000002000000000000000000000000000000000000000000000000000000000000000000000000000000000000000000000000000000000000000000000000000000000000000000000000000000000048000000000000000000010FD00
:5C8FC000000040010000000000004000000000000000000000014A0000000000800000000000000000000000000000000000000000000000000000000000000000000000004000000000000000000002400000000000000000000040000038FF10
:5C901C00000000008000000000000000000000000000000000000000000000000000000000000000000000000000000000000000000000000000000000000000000000000000000000000000000000000000000000000000000000000000D4FFA5
:5C907800000000000000000000000000000000000000000000000000000000000000000000000000000000000000000000000000000000000000000000000000000000000000000000000000000000000000000000000000000000000000DCFFC1
:5C90D400000000000000000000000000000000000000000000000000000000000000000000000000000000000000000000000000000000000000000000000000000000000000000000000000000000000000000000000000000000000000DCFF65
:5C9130000000000000000000000000000000000000000000004000000000000000000000004000800000000000000000000000000000000000000000000000000000000000000000000000000000000000000800000200000000000000007CFD60
:5C918C0000000008000000000000000080000000000000000200000000000000000000000000010000000000000000000000000000000000000000000000000000000000004000000000000000000000000000000000000000000010000020FE8E
:5C91E80000001000000000000008000000000000000000001400000000000000000000000000000000000000000000000000000000000000000000000000000000000000000000000000000000000000000000002000000000000010000084FD4E
:5C92440000000410000200000000012040000000000000400008000500000000000000000000080000000000000000000000000000000000000000000000000000000000000000000000000000000000280004A000000000000000400000FCFCFE
:5C92A00000000480000000004000080001000000000010000200000000000000000000000002000000000000000000000000001000000000000000000000000000000000002800000000000000100000000000000100000000001000000050FFE9
:5C92FC00000000002000000000000000400000000100100000400000000020000001000004000010000000000000000000000000000000000000002000008000000400000000000000000000000000000000080000000000000000000000D8FDAF
:5C93580000000000000800000000000000100000400000000000000000000000004000000001000004000000000000000000000000000000002000000000000000000100000000000000000000000000000000000000000000000000000008FDF6
:5C93B4000000008001000000000000000300000C0000300001C00000000060000C0000300000C000000000000000000000000000000000001800006000008001300000000000000000000000000000000000180000000000000000000000B8FF88
:5C941000000000800000000000000000010000040000D0020040000000002000040000100000400000000000000000000000000000000000080000200000800010000000000000000000000000000000000008000000000000000000000030FD08
:5C946C000000000046010000000000008C020030210000020000230000008081300000C028000013000000000000000000000000000000006020008041000046C0880000000000000000000000000000000060440000000000000000000098FE24
:5C94C8000000000007000000000000000E0000380000E020008083000000C001382000E00000808300000000000000000000000000000000700000C001000007E10000000000000000000000000000000000700000000000000000000000E4FF90
:5C9524000000000006000000000000000C0000300000C0800000030000008001300000C000000003000000000000000000000000000000006000008001000006C0000000000000000000000000000000000060000000000000000000000004FEE9
:5C9580000000000006000000000000000C0000300000C0000000030000008001300000C000000003000000000000000000000000000000006000008001000006C000000000000000000000000000000000006000000000000000000000000CFE05
:5C95DC0004000000001000000000000040000030820000040040000000400008040000000000001000000000000000000000000000000000600400000000800000040200000800010000008000000000004300000000000001001000008022FC28
:5C96380000000000000000000000000000100000400000000100000000001000020000000000000004000000000000000000000000000000008000000000000000000100000000000080000000000000000000000000000040000000000084FDAD
:5C9694000800000000300000000000000300003C8001300000C00000000360000C1000000000C00000000000000000000000000000000000788000000000800130000600001800037000008001000000C08300000000000C000030000000F1FE2A
:5C96F000000000000010000000000000010000B4A000100000400000000120003402000000004000000000000000000000000000000000006801000000008000100002000008002D20000080000000004023000000000004000010000080DDFC32
:5C974C000400000000C00800000000008C1000300AC6C02200000300002C80210040000000000013040000000000000000000000000000006002000000000046C400180500600280800901002604000000230000000000300200C040000011FFCC
:5C97A8000000000000E00001000000000E0000380007E00000800302000EC8013800000000008003000000000000000000000000000000007080000000000007E0801C000070200EC40100000700000080030400000000382000E000000090FD17
:5C9804000800000000C00000000000000C0000300806C00000000300000C80013008000000000003000000000000000000000000000000006010000000000006C00018000060000C800100000600000000830000000000300000C000008014FE25
:5C9860000000000000C00000000000000C0000300206C00000000300000C80013002000000000003000000000000000000000000000000006004000000000006C00018000060002C8401000006000000000B0000000000300000C000000094FF3C
:5C98BC00040000000010000000000000010000308200C00800001000008C2000300200C01000001000000000000000000000000000800000080000000000002010000200000000000000000020000000000000000000000001001000008078FF11
:5C99180000000000000000000000000000000000400000000100000400001000004000000000000004000000000000000000000000002000000000000000000008000000000000000080000000080000000000000000000040000000000088FCE6
:5C9974000800000000300000000000000304003C8001F00000C00000000F60003C0000F00000C00000000000000000000000000000060000180000000000800130000700000000006000008001000000000000000000000C00003000000079FC28
:5C99D0000000000000100000000000008D0000348900D02000400000000D2200340900D080004000000000000000000000000000000200000800000000008000D0020200000000002000008000000000000000000000000400001000000064FE41
:5C9A2C000400000000C0240000000000400000B00846C00400002300004C8201301200C0240000130000000000000000000000000018010060400000000000460000590800000000800500004601000000000000000000302100C008008040FCC8
:5C9A88000000000000E00000000000000E0200380007E12000800301000EC001390000E000008003020000000000000000000000001C08007000000000000007E1001C0000000000C08100000700000000000000000000380000E020000084FDC8
:5C9AE4000800000000C00000000000000C0000301006C04000000300000C8001302000C080000003000000000000000000000000001800006000000000000006C020180000000000800100000600000000000000000000300000C00000009DFC63
:5C9B40000000000000C00000000000000C0400300006C00200000300008C8201300200C000000003000000000000000000000000001800006000000000000006C002180000000000800100000600000000000000000000300000C000000074FCBB
:5C9B9C000400008000000400000000008C0000040020000400400000004000080400000000004000000000000000000000000000008000000800000000000020C0088000000000008021000020000000000000000000000400000004008088FEA6
:5C9BF80000000000000000010000000000100000000008000100000000001000020000000000000000000000000000000000000000002000000000000000000008000120000000000000000000080000000000000000000000000000010064FF30
:5C9C54000800008001300000000000000F00000CC001300000C00000000360000C1000000000C000000000000000000000000000000600001800000000008001F000060000000000E001008001000000000000000000000C000030000000CDFDF3
:5C9CB0000000008000100000000000008D0800B48000100000400000000120003402000000004000000000000000000000000000000200000800000000008000D020020000000000A0450080000000000000000000000004000010000000B0FD76
:5C9D0C000400000026C82400000000008C0000000226C04000000300008C80410006000000000023000000000000000000000000001803006001000000000016C000580000000000801100004600000000000000000000300900C0020080D8FFE5
:5C9D68000000000007E00000000000000E0200380807E20000808300000EC8013800000000008003010000000000000000000000001C00007010000000000007E8201C0400000000C04100000701000000000000000000380000E0200000A0FC41
:5C9DC4000800000006C00000000000000C0200300006C00000000300000C80013008000000000003000000000000000000000000001800006000000000000006C020180000000000804100000600000000000000000000300000C000000089FFF1
:5C9E20000000000006C00000000000002C0000301106C00000000300000C80013000000000000003000000000000000000000000001800006000000000000006C004180000000000800100000600000000000000000000300000C000000004FE57
:5C9E7C000400008000100002400000008C000000018610000000100000400008040000000400001000000000000000000000000000800000000000000000012010000200000000002000000020000000001000000000000480000004008024FDF5
:5C9ED8000000000000000000000000000010000040000000000000040000100002000000000100000400000000000000000000000000200000200000000040000800000000000000000000000008000000000400000000000000000001001CFD15
:5C9F34000800008001300006C00000000F00000C8007300000C00000000360000C1000300000C0000000000000000000000000000006000018000000000C800130000600000000006000028001000000C00000000000000C80013800000049FEC1
:5C9F90000000008000100002400000002D10000480461100004000000001200034020010000040000000000000000000000000000002000008000000000480001000020000000000A00500800000000040000000000000048016100000002CFFCA
:5C9FEC000400000026C00898100B00000C0000302246C12200002300002C8205804000C0220000A30000000000000000000000000058040060020000003000160042580000000000000800000601000000A300000000003001C0C002018014FE3C
:5CA048000000000007E1201C800302000E0200380007E00000808300000EC041380000E000008003000000000000000000000000001C0000701000000038200724001C0400000000C04100000700000080030000000000384007E000000048FFC7
:5CA0A4000800000006C00018000300000C0000300006C20000000300000C8001300800C000000003000000000000000000000000001800006000000000300006C000190000000000800100000600000000030000000000300006C100000029FDBA
:5CA100000000000006C00018000300004C0800300046C00000000300000C8001B00000C000000003000000000000000000000000001800006000000000300006C002180000000000800102000600000000030000000000300026C000000034FC3B
:5CA15C0000000000201000000010000040000000012010000000100000018011040000100000002300000000000000000000001000020000600400200000014610008000000000002000000046000002001000000000000480000004000038FC7C
:5CA1B80000000000000800000000040000100000400008000000000400000000020000000000000004000000000000000000000000000000008000000000400008000020000000000000000000080000000004000000000000000000010068FD83
:5CA214000000008001300000C00000000300000C8001300000C000000003E0010C1000300000C0030000000000000000000000300006000078000060000C800730000700000000006000028007000006C00000000000000C800138000000A0FF1F
:5CA270000800008000100000400000000100000480001000004000000001A0413402001000004083000000000000000000000010000200006812002000048046D102020000000000A0050080460100024000000000000004801610000000C9FF8F
:5CA2CC000000000026C00200009300002C1000B02046C00200000300008C8151800000C0280000030000000000000000000000C00258200060020080013001460104980400000000000001001600009810230000000000300110C00800007CFE41
:5CA328000000000007E12000800300000E0000380007E10001808300000EC001380800E0000080830000000000000000000000E0801C0000702000C041381007E0201C0000000000C00100000701001C80030200000000380807E22000002CFCD7
:5CA384000400000006C00000000300000C0000300006C00000000300000C8041300000C0000000830000000000000000000000C0001800006010008001300006C120180000000000804100000601001800030000000000300006C1000080E0FC3D
:5CA3E0000000000006C00000000300000C0000300006C00000000300000C8011300A00C0000000230000000000000000000000C0001800006000008001300046C008180000000000801100004600001800030000000000300046C0000000ECFD79
:5CA43C00240000800000040040000800010000000120100000001000000100080400201000004000000000000000000000000000001801000000000000000120100002000000000000000080000000004000000001200000810010000080C4FE15
:5CA49800000000000000000100000000000000004000080000000004000000000200000800000000000000000000000000000000000020000020000000004000080000000000000000800000000000000000000000000000400000000000D4FCF9
:5CA4F4006800008001300000C00018000300000C8001300001C00000000360000C8001300000C000000000000000000000000000001E000018000000000C800130000700000000006000008001000000C00000000360000C800138000000C9FE30
:5CA55000200000800010000040000800010000048000D00200400000000120000480001000004000000000000000000000000000001A05000800000000048000D0020200000000002000008000000000400000000120000480161000000070FE93
:5CA5AC008481000046C40200009360028C100030104600040100230000208001000146C00800002300000000000000000000000000580000600100000030020600489804000000008009000046000000000300008C8011301210C202008084FC56
:5CA60800C001000007E02000800370200E0000380007E800008003020002C241081007E800018003020000000000000000000000001C04007010000000384007E1001C0000000000C001020007040000800302000EC4013A0007E0200000F4FE5A
:5CA664008801000006C00000000360000C0000300006C00000000300000C9001301006C000000003000000000000000000000000001804006000000000300006C0001800000000008001000006000000000300000C8001300006C100000081FE26
:5CA6C0008001000006C00000000360000C0000300006C08400000300002C8001300206C000000003000000000000000000000000001801006000000000300006C0221800000000008001000006000000000300000C8001300016C0000000A4FCFD
:5CA71C000000048000000400400000000120000400201000020023000001200004000010008000230000012000040000000000000002400008000120003084000004804000080001200004800010000040000000012000B08800C0080280C4FD5E
:5CA7780000000000000000010000000000000000000008000000000400000000000000000000200004000000000000000000000000000000000000000000000000000120000000000000000000000000000000000000000000000000010080FDB5
:5CA7D40000000C8001300000C00000000364000CC001300007C08300000360000C1000300006C00300000360000C0000000000000006C00018000360003C8801300006C00018000360000C8001300000C00000000360003C8001F0000600B5FC5C
:5CA830000C00048000100000400000008D2000B48000D00202400B0000012000340200100002408B0000012000040000000000000002400008000120003480001000024000080001200004800010000040000000012000B48800D028020038FC9A
:5CA88C000400B00046C10800000B0400408291800016000818010B00002C8205020200C02218004300002C8009301000000000000058041361022C8009300906C01018054360024C8405324246C2000000A300002C8411300240C0021889CCFFF3
:5CA8E8000000384007E02000800300000EC001380807E1801C908300000EC001381000E0001C900300000EC80139000000000000001C800370100EC481380007E1001C800370800EC001380007E08000800300000EC001390801E4801C00ACFC6B
:5CA944000400300006C00000000300000C8001300006C00018008300000C8001300000C00018000304000C8001300000000000000018000360000C8001300806C00018000360000C8001300006C00000000300000C8001300806C8201800B9FFB9
:5CA9A0000000300006C00000000300002C8201300A06C02418000300000C8001300800C00018000300000C8001300000000000000018000360000C8001B00006C00018000360000C8001300006C00000000300000C8001300016C008180054FD94
:5CA9FC0004000000000000000000000000000000000000000000000000000000000000000000000000000000000000000000000000000000000000000000000000000000000000000000000000000000000000000000000000000000008050FF2C
:5CAA5800200004800010000240000800012000048000100002400008000120000480001000024000080001200004000000000010000240000800012000048000100002400008000120000480001000024000080001200004800010000200BCFCBA
:5CAAB400080000000000000000000000000000000000000000000000000000000000000000000000000000000000000000000000000000000000000000000000000000000000000000000000000000000000000000000000000000000000C5FE7B
:5CAB1000200004800010000240000800012000048000100002400008000120000480001000024000080001200004000000000010000240000800012000048000100002400008000120000480001000024000080001200004800010000200BCFC01
:5CAB6C00040120000480001000024000080001200004800010000200000800012000048000100002000008000120000000000080001000024000080001200004800010000240000800012000048000100002400008000120000480001080CCFD15
:5CABC80000000000000000000000000000000000000000000000000800000000000000000000000008000000000000000000000000000000000000000000000000000000000000000000000000000000000000000000000000000000000054FFCE
:5CAC2400880010000240000800012000048000100002400008000100000480001000024000080001000004800010000000000040000800012000048000100002400008000120000480001000024000080001200004800010000240000800A9FD94
:5CAC800000000000000000000000000000000000000000000000000800000000000000000000000008000000000000000000000000000000000000000000000000000000000000000000000000000000000000000000000000000000000054FF15
:5CACDC00000000000000000000000000000000000000000000000000000000000000000000000000000000000000000000000000000000000000000000000000000000000000000000000000000000000000000000000000000000000000DCFF41
:5CAD3800000000000000000000000000000000000000000000000000000000000000000000000000000000000000000000000000000000000000000000000000000000000000000000000000000000000000000000000000000000000000DCFFE4
:5CAD9400000000000000000000000000000000000000000000000000000000000000000000000000000000000000000000000000000000000000000000000000000000000000000000000000000000000000000000000000000000000000FEFD68
:5CADF000000000000000000000000000000000000000000000000000000000000000000000000000000000000000000000000000000000000000000000000000000000000000000000000000000000000000000000000000000000000000DCFF2C
:5CAE4C0000000000000000000000000000000000000000000000000000000000000000000000000000000000000000000000000000000000000000000000000000000000000000000000000000000000000004000000000080000000000058FFCF
:5CAEA800000000000000000000000000000100000000000000000000000000000000000000000000010000000000000000000000000000000000000000000000000000000000000000000000000000000000000000000000000000000000CCFF81
:5CAF0400000000000000000000000000000000000000000000000000000000000000000000000000000000000000000000000000000000000001000000000000000000000000000000000000000000000000000000000000000000000000CCFF25
:5CAF6000000000000000000000000000000000000000000000000000000000000000000000000000000000000000000000000000000000000000000000000000000000000000000000000000000000000000000000000000000000000000DCFFBA
:5CAFBC00000000000000000000000000000000000000000000000000000000000000000000000000000000000000000000000000000000000000000000000000000000000000000000000000000000000000000000000000000000000000DCFF5E
:5CB01800000000000000000000000000000000000000000000000000000000000000000000000000000000000000000000000000000000000000000000000000000000000000000000000000000000000000000000000000000000000000DCFF01
:5CB07400000000000000000000000000000000000000000000000000000000000000000000000000000000000000000000000000000000000000000000000000002000000000000000000000000000000000000000000000000000000000FCFD67
:5CB0D00000000000000000000000000000000000000000000000000000000000080100000000000000000000000000000000000000000000000000000000000000000000000000000000000000000000000000000000000000000000000044FFD8
:5CB12C00020000000000000000000000000000000000000000000000000000000000000000000000000000000000000000000000000000000000000000000000000000000000000000000000000000000000000000000000000000000000FCFDCC
:5CB18800000000000000000000000000000000000000000000000000000000000000000000000000000000000000000000000000000000000000000000000000000000000000000000000000000000000000000100000000000000000000FEFC70
:5CB1E400000000000001000000000000000000000000000000000000000000001000004020000000000000000000000000000000000000000000000200000002000000000000000000400000000000000000001000000000000000000000A8FFA3
:5CB24000000000000000000000000000000000000000000000000000000000000000000000000000000000000000000000000000000000000000000000000000000000000000000000000000000000000000000000000000000000000000DCFFD7
:5CB29C00000000000002000000000000000000000000000000000000000000000800002040000000000000000000000000000000000000000000000400000001000000000000000000800000000000000050002000000000000000000000A0FE59
:5CB2F800000000000040000000000000000000000000000000000100000000008000000000000000000008800000000000000000000000000010400000000000002808002002000000080000000000000010000200000000000000000002D0FC27
:5CB3540000000000004000000000000000000000000000000000010000000000000000000000000000000000010000000000000000000000001000000000000000200800000000000000000000000000000000000000000000000000000038FCEF
:5CB3B0000000000000000000000000000000000000000000000000000000000000000000000000000000080000000000000000000000000000000000000000000000000000000000000000000000000000000000000000000000000000105CFECF
:5CB40C00000000000000000000000000000000000000000000000000000000000000000000000000000000000000000000000000000000000000000000000000000000000000000000000000000000000000000000000000000000000000DCFF09
:5CB46800000000000000000000000000000000000000000000000000000000000000000000000000000000000000000000000000000000000000000000000000000000000000000000000000000000000000000000000000000000000000DCFFAD
:5CB4C4000000000000000000000000000000000000000000000000000000000000100000000000000000000000000000000000000000000040000000000000000000000000000000000000000000000000400000000000000000000000009CFE02
:5CB5200000000000000000000000000000000000000000000000000000000000000000000000000000008000000000000000000000000000000000000000000000000000000000000000000000000000000000000000000000000000000054FFFC
:5CB57C00000000000000000000000000000000000000000000000000000000000000000000000000000000000000000000000000000000000000000000000000000000000000000000000000000000000000000000000000000000000000DCFF98
:5CB5D800000000000000000000000000000000000000000000000000000000000000000000000000000000000000000000000000000000000000000000000000000000000000000000000000000000000000000000000000000000000000DCFF3C
:5CB63400000000000000000000000000000000000000000000000000000000000000000000000000000000000000000000000000000000000000000000000000000000000000000000000000000000000000000000000000000000000000DCFFDF
:5CB69000000000000000000000000000000000000000000000000000000000000000000000000000000000000000000000000000000000000000000000000000000000000000000000000000000000000000000000000000000000000000DCFF83
:5CB6EC00000000000000000000000000000000000000000000000000000000000000000000000000000000000000000000000000002000000000000000000000000000000000000000000000000000000000000010000000000000000000FCFCDA
:5CB74800000000000000000000000000000000080000000000000000000000000000000000000000000000000000000000000000000000000000000000000000000000000000000000000000000000000000000000000000000000000000D4FFCA
:5CB7A400000000000000000000000000000000000000000000000000000000000000000000000000000000000000000000000000000000000000000000000000000000000000000000000000000000000000000000000000000000000000DCFF6E
:5CB80000000000200000000000000000000000000000000000000000000000000000000000000000000000000000000000000000000000000000000000000000000000000000000000000000000000000000000000000000000000000000FCFFD1
:5CB85C0040000000000000000000000000040000000000000000000000000080000000000000000000000000000000000000000000000000000000000000000000000000000000000000020000000000000000000400000000000000000018FDB1
:5CB8B800000000000000000000000000000000000000000000000000000000000000000000000000000000000000000000000000000000010000080000000000000000000000000000010000000000000000000000000000000000000000D4FF57
:5CB9140000000000000000000000000000000008010040000002040000000100200800000000002400000000100800000000000000000800100000000120000040000000000000000000000000000000000000000000000000002040000030FE1C
:5CB970000000000000000000002000000048000000020000000000000080000000000000000000000000000000000000000000000000000000000000000004001000000000000008000000000100100000000000000000080000000800001CFF39
:5CB9CC000000000000000000000000000000000000002000000000000001400000000000000000000000000000000000000000000000000000000000000000000000080000404000000001000000000000000000000020000000000000001CFDFC
:5CBA280000000000000000000000000000000000000000800000000000000000000000000000000000000000000000000000000000000000000000000000000004000040000000040000000800000000000000000000000000000000040010FFDF
:5CBA8400000000000000000000000000000000000000000000000000000000000000000000000000000000000000000000000000000000000000000000000000000000000000000000000000000000000000000000000000000000000000DCFF8B
:5CBAE000000000000000000000000000000000000000005000000000000000000000000000000000000000000000000000000000000000000000000000000000000000000000000000000000000000000000000000000000000000000000C8FEF4
:5CBB3C00000000000000000100004000000000000004000000004000000000004000000800000040000000000000000000000000000000000000000000000000000000000000001000000000800000000000000000000000040200000000C0FD4D
:5CBB980000000000000000000000000000000040000000000000400000000000000400000200408000000000000000000000000000000000000000000000001000120000000000000000000000000000004000000000000000040000000064FD44
:5CBBF4001C00000000000000000000000000000000000000000000000000000000000000000000000000000000000000000000000000000000000000000000000000000000000000000000000000000000000000000000000000000000C01DFEFE
:5CBC5000000000000000000000000000000000000000000000000000000000000000000000000000000000000000000000000000000000000000000000000000000000000000000000000000000000000000000000000000000000000000DCFFBD
:5CBCAC0000000000004120000001200000000000000001200000810000040000000000000000000000000000001000000000000000080000000000800000000020000000000000000000000000000008000000000400000000020000080084FDC5
:5CBD0800000000000000000000000000000000100000000000000000000000000000000000000000000000000000000000000000000044000000000000000000400000000000000100000000000000000000000000000010000040000000CCFF2F
:5CBD6400000000000022400080001000000000040014024000800001000200000000000000000000000000000008000000000000000450004001004000000000300000000020000180000000140000040000000002000004000110000400C8FF0C
:5CBDC000800200220440242205069000000000A00012210000000900000420420000024028080081000004000090080000000000009000A50001940204100A04000008040020010020240004920000400402200021C0708024105021400000FF7D
:5CBE1C008000000000402000040000000000000000020100000001000004004000000140200800810000040000102000000000000000008100000402001008000000080400200000000000800000000004000800002000010000802000007CFCF0
:5CBE780000000000020000000001000000000010000000000000000000000000000000000000000000000000000000000000000000080000000000000000000200000000000000000040000400010000000100000000400008000000000068FD5E
:5CBED4000000000000048000000002000008000020000480000000020000080001200004800010000200000000000000000000000000100000000000000020000480001000000000000000000004000000000200000000002000008000001CFE9B
:5CBF30000A00000000020000000000000000000000000000000000000000002000000000000002000000000000000000000000000000000080000000000000000000000000000000000200000000000000000000000000000000000000C001FC48
:5CBF8C0000000000000000000000000000000000000008000000000000000000000000001001000000000000000000000000000000000000004000000000000000000000000000000004000000000000000000000000000000000000000084FF79
:5CBFE80000000000100000800000000000000080010000000000000000000000000000000000000000000000000000000000000000000000000000000000000020000000000000000000000020000000000000000000000001000000000054FE59
:5CC04400000000000000000000000000000000000000000000000000000000000000000000000000000000000000000000000000000000000000000000000000000000000000000000000000000000000000000000000000000000000000DCFFC5
:5CC0A000000000000000000000000000000200000000000200000000000000000000000000000000000000000000000000000000000000000000000000000000000000000000000000000000000000000000000000000000000000000000DCFF65
:5CC0FC00000000000000000000000000100000000000000000000000000000000000000000000000000000000000000000000000000000000000000000000000000000000000000000000000000000000000000000000000000000000000CCFF0D
:5CC15800000000000000000000000000000000000000000000000000000000000000000000000000000000000000000000000000000000000000000000000000000000000000000000000000000000000000000000000000000000000000DCFFB0
:5CC1B40000000000000000000000000080000000000000100000000000000000040000000000000000000000000000000000000000000000002000000000400000000000000000000000000000000000000000000000000200800000000024FC99
:5CC2100000000000000000000000000000000000020000000000000000002000000000000000000000000000000000000000000008000000000000000000004000000000000000000000000000000000000000000000000000000000000090FFD9
:5CC26C0000000000000000000000010000100000D00000400100000400001400024000000000000004000000000000000000000000022000008000000000000008400100000000000480000000080000000000000000000000000200010078FC08
:5CC2C80000000000000000000000000004000000800000000000000000000000100000100000000000000000000000000000000000000000000000000004000000000000000000002008000000000080400000000000000000000000000058FD35
:5CC32400200004000000000000000002000008000000000080001000004000000000000000000010000000000000000000000000000000000002000000300200000000000000000000000000200000000043000000000000000000008000CCFDCF
:5CC3800000000000000000000000008000000002000000000020000400001000000000000000000004000000000000000000000000000000008000000000400000000000000000000000000000080000000000000000000000000000002014FEAD
:5CC3DC0060000C000000000000001800006000000000000006C0000000030000000000000000C0000000000000000000000000000000000018000000003C000000000000000000000000008001000000C00300000000000000000000060028FDD5
:5CC4380020000400000000000000080000200000000000000240000000010000000000000000400000000000000000000000000000000000080000000034200000000000000000000000008000000000401302000000000000000000020070FF37
:5CC494008011B0000000000000006002008081000000000018009300008C1000000000000000000B00000000000000000000000000000000601100000030010000000000000000000000000026040000008B0000000000000000000058105CFC3F
:5CC4F000C0413808000000000000701000C00100000000001C900300000E00000000000000008003040000000000000000000000000000007000000000381000000000000000000000000000070000008003000000000000000000001C00D4FFF9
:5CC54C00800130000000000000006000008001000000000018000300000C0000000000000000000300000000000000000000000000000000600000000030000000000000000000000000000006000000000300000000000000000000180084FCA6
:5CC5A800800130000000000000006000008001000000000018000300000C00000000000000000003000000000000000000000000000000006000000000B0100000000000000000000000000006000000004300000000000000000000180050FDAD
:5CC604002400000100000000000000020000080400000000020010000001000000000000008000100000000000000000000000000000000000020000003002001000000000600400200004002000000040000800000000040000000080009CFDB3
:5CC66000000000400000000000000080000000020000000000000004000000000000000000002000040000000000000000000000000000000080000000004000000000000000800000000000000800000000000000000000000000000020D4FD5B
:5CC6BC0068000C0000000000000018000060000C0000000006C0000000031000000000000006C0000000000000000000000000000000000018000000003C1000300000000078000060000C8001000000C00019000000000C0000000006009CFF0C
:5CC71800200004000000000000000800002000040000000002400000002D00000000000000024000000000000000000000000000000000000800000000340100100000000068400020000480000000004023080000000004000000000280A8FD95
:5CC77400840931060000000000006011008011300900000058001300002000000000000000981023020000000000000000000000000000006084000000304200C000010000600200804530222608000000086041000000B008000000188145FC19
:5CC7D000C0013800000000000000700000C0013A000000001CA08300000E040000000000001C8003000000000000000000000000000000007000000000380000E000000000701000C0013800070000008083700000000038000000001C0898FF4B
:5CC82C00880130000000000000006000008001300000000018000300000C00000000000000180003000000000000000000000000000000006000000000304000C00000000060000080013000060000000003600000000030000000001800FDFE57
:5CC88800800130000000000000006000008001300000000018000300004C01000000000000180003000000000000000000000000000000006000000000300200C000000000601100800130000600000000A36000000000300000000018007CFED0
:5CC8E400200004000000000000000002018021000100100080000000008C00000000000000184100000000000000000000000000000000000800000000300200000400000000020020000400200000000043080000200004000000001801F8FFB7
:5CC940000000000000000000000000800000000040000000002000000000100000000000000020000000000000000000000000000000000000000000000040000000010000008000000000000008000000000000000000000000000000204CFE58
:5CC99C0060000E00000000000000180003E0410C0000300006000000000F020000000000001EC4000400000000000000000000000000000018200000003C0000300000000018000060000C8001000000C00318000060000C000000001E0450FCFE
:5CC9F800A8050400000000000000080001A001040000100002000000002D000000000000001A400B0000000000000000000000000000000068040000003404001000000000080000200004800000000040030C0000200004000000001A0095FE60
:5CCA54000008300100000000000060108C8805300A00C00218010000000C00000000000000180190000000000000000000000000000000000041000000302200C0240000006080008011300246010000009360020080113202000000180080FC4B
:5CCAB000C041380800000000000070000EC001390000E0001D040000000E080000000000001C8403000000000000000000000000000000007000000000380000E000000000700000C0413808070000008003701000C00138080000001C0410FD46
:5CCB0C008401300000000000000060000C8001300000C00018000000000C04000000000000180083000000000000000000000000000000006080000000300000C0000000006000008001300006000000000360000080013000000000188420FDC4
:5CCB68008009320000000000000060000C8049300000C00018000000004C00000000000000180503000000000000000000000000000000006002000000B02000C0000000006000008001300006000000002361000080013000000000180100FDB9
:5CCBC400841104000000000000000800408021000100000002400000008C0000000000000080002300000020000000000000000000000000600400000004000010000000000002000008040046000000400008000000080001000000800008FD5F
:5CCC20000000020000000000000000000010000040000000000000000000100000000000000020000400000000000000000000000000000000800000000000000000000000008000000002000008000000000000000000024000000000202CFD9D
:5CCC7C00E8010C00000000000000180003E0010C0000000006C00000000F0000000000000006C0030000006000000000000000000000000078000000000C1000300000000018000060000C8007000000C00019000060000C000000000600BCFE8D
:5CCCD800A0050500000000000000080001A001050000000002400000002D0800000000000002408300000020000000000000000000000000681000000034020010000000000800002000048006010000402308000020000400000000028058FD74
:5CCD34008451300200000000000060102C8209300900000018010300000C00000000000000182103000000800900000000000000000000006000000000000000C0080000006012008045B0000600000000006004008089B008000000188175FF08
:5CCD9000C001384000000000000070000EC00139000000001C840302000E020000000000001C8083000000C00101000000000000000000007010000000380800E080000000700000C0013808070100008083701000C00138000000001C10B0FE11
:5CCDEC008801300000000000000060000C8001300000000018000300000C04000000000000180083000000800100000000000000000000006010000000300800C00000000060000080013000060000000003600000800130000000001800B5FF6F
:5CCE48008011320000000000000060000C8041300000000018000300000C0000000000000018000B000000800100000000000000000000006004000000B00000C00000000060000080013000160100000023620000800130000000001800E8FF72
:5CCEA400841100010000000000000800402000040000000002400000000100000000000000020023000000000800000000000000000000000002000000040000100000001008000000080081000000000010000200000800010000008000E8FE88
:5CCF000000000240000000000000000000100000000000000000000000000000000000000000000004000000000200000000000000000000008000000000000000000000000400000000024000000000000004800000000240000000002068FE6B
:5CCF5C00E8810C0000000000000018000360800C0000000006C0000000031000000000000006C0030400006000000000000000000000000018000000000C1000300000C00018000060000C8001000000C00018000060000C0000000006003CFE4A
:5CCFB800A0090400000000000000080001A011040000000002400000002D00000000000000024023000000200000000000000000000000000800000000340200100000400008000020000480000000004000080000200004000000000280ECFDAD
:5CD014008445300100000000000060022C0004300A00000018011300004000000000000000180083000000805100000000000000000000006020000000800000C008000003608100801130020600000000A3600200800530020000001891C1FF88
:5CD07000C001380800000000000070100EC24138000000001C888300000E020000000000001C9003000000C00100000000000000000000007000000000380800E040008003740000C0413808070800008003701000C04138080000001C0080FFFD
:5CD0CC008801300000000000000060000C8041300000000018000300000C00000000000000180003000000800100000000000000000000006000000000300000C00000000360000080013000060000000003600000800130000000001800B1FDEB
:5CD128008029300000000000000060000C8005300000000018000300000C0200000000000018000B010000800100000000000000000000006000000000300A00C000000003600000800130000600000000036000008001300000000018003CFD0A
:5CD18400040000010000000000000800012000040000000018011000004000000480001000020010000000000800000000000010000000000800000000040000000400000008000020000001200000000010000200000804000000008080B4FECD
:5CD1E00000800040000000000000000000000000000000000020000400001000000000000000000004000000000200000000000000000000000000000000000000000100000000000000004000080000000004800000000200000000002020FCEE
:5CD23C0068000C0000000000000018000360000C000000001EC40000000300000C8001300006C0000000006000000000000000300000000018000000000C1000300000000018000060000C8001000000C00018000060000C00000000060039FFB8
:5CD2980020000400000000000000080001200004000000001A400000000100000480001000024000000000200000000000000010000000000800000000340200100000000008000020000480000000004000080000200004000000000200B4FC70
:5CD2F4008401B00000000000000060802C0004320200000018008300002C0800304246C2184000030400008009000000000000C0400000006042000000000200C0040000000004008011300126010000000B6004008051300600000018A0F0FFC2
:5CD35000C041380800000000000070000E420038080000001C840300000E0000380007E000048403000000C041000000000000E0000000007000000000380800E020000000101000C0813808070000008003711000C00138000000001C00B4FDE2
:5CD3AC008801300000000000000060000C8081300000000018000300000C0000300006C0001820030000008001000000000000C0000000006000000000300800C0000000006020008001300006000000000360000080013000000000180021FD5D
:5CD408008001300000000000000060000C8011300000000058040300000C0000300006C0005800030000008001000000000000C0000000006000000000300000C000000000600400800130000600000000036000008001300000000018003CFF1B
:5CD4640004003004000000000000000201000804800000008040000000010000008000000080400000000020000000000000000000000000080000000004000000040000000800010008008100000000400000020020000081000000808068FE99
:5CD4C00000800000000000000000008000000002000000000020000000000000000000000000200000000000000000000000000000000000000000000000000000000100000000000000024000000000000000800000000040000000002060FF4C
:5CD51C0068003C0000000000000018000360000C8001000006C0000000031000008001000006C0000400006000000000000000000000000018200000000C0000300000000018000360000C8001000000C00018000060000C800100000600CDFD72
:5CD57800200034120000000000000800012000048000000002400000002D0000008000000002400B000000200000000000000000000000006804000000040000100000000008000120000480000000004000080000200004800000000200D0FFFE
:5CD5D4008411300200000000000060122C8201324086000098049300004000000000260400980410000000800502000000000000000000000002000000002100C00800000060124C9005B00026010000000B6001008009B1001600001882BCFE2A
:5CD63000C041380800000000000070000EC00138000700001C800300000E040000000700001C8083000000C00100000000000000000000007010000000080000E02000000070000EC0413808070000008003711000C00138080702001C0014FEBD
:5CD68C008801300800000000000060000C8001300006000018000300000C04000000060000180003010000800100000000000000000000006000000000301000C00000000060000C8001300006000000000360000080013000060000180071FE6C
:5CD6E8008001300200000000000060000C8001300006000018000300008C00000000060000180003000000800100000000000000000000006011000000300200C00000000060000C8001300006000000000360000080013000060000180018FEF9
:5CD74400200000010000000000000800012000000100000002400008000100080080000000020010000000801100000000000000000000000800010000040000C0080000000800002000048000100000400008000080110400001000180158FCDD
:5CD7A0000000004000000000000000000000000040000000000000000000000002000000000000000400000000020000000000000000000000000000000000000000010000000000000000000000000000000000000000020000000000208CFFF7
:5CD7FC0060000E0000000000000018000364800C0000000006C0001800037000008001000006C000000000E041000000000000000000000018000304000C1000F02000000018200060000C8001300000C000180000E0410C000030001E042CFD7F
:5CD85800A805040000000000000008008DA011040000000002400008002D20000080000000024000000000A011000000000000000000000008008D0000340200D00000000068040020000480001000004000080000A01104000010005A00D5FE7A
:5CD8B400004830000000000000006011200808300200000098042364202080050200160200980413020000804500000000000000000000006011000400802000C002000000000C008005300146C1000100A36001008009B00000C004180130FF6B
:5CD91000C001380800000000000070000EC04138080000001C800370000EC20100000700001C8003000000C001000000000000000000000070000E0000380000E020000000700000C041380807E000008003701000C041380800E0401C049CFF47
:5CD96C008401300000000000000060000C9041300000000018000360000C820100000600001800030000008081000000000000000000000060000C0000300800C0200000006080008001300006C0000000036000008041300000C000188004FD89
:5CD9C8008045300000000000000060002C8011300000000018000360008C800100000600001800030000008011000000000000000000000060004C1000300200C0020000006000008001300006C0000000036000008005300000C0001805E4FF28
:5CDA240000000000000000000000000000000000000000000000000000000000000000000000000000000000000000000000000000000000000000000000000000000000000000000000000000000000000000000000000000000000008076FDB3
:5CDA8000200004800010000240000800012000048000100002400008000120000480001000024000080001200004000000000010000240000800012000048000100002400008000120000480001000024000080001200004800010000200BCFC62
:5CDADC00000000000000000000000000000000000000000000000000000000000000000000000000000000000000000000000000000000000000000000000000000000000000000000000000000000000000000000000000000000000000CDFE23
:5CDB38002C000480001000024000080001200004800010000240000800012000048000100002400008000120000400000000001000024000080001200004800010000240000800012000048000100002400008000120000480001000028029FDAF
:5CDB94000401200000000000000040000800012000048000100002400008000120000480001000020000000001000000000000800000000040000800002000008000000002400008000120000480000000024000000001200004800010009DFF27
:5CDBF0000000008000100002400000000000000000000000000000000000000000000000000000000800010000040000000000000002400000000020000080000000020000000000000000000000000200000000010000000000000000003CFED9
:5CDC4C00840010000000000000002000048000100002400008000120000480001000024000080001000000800000000000000040000000002000040000100000400000000120000480001000024000000001200000800010000240000880D8FD6F
:5CDCA8000000008000100002400000000000000000000000000000000000000000000000000000000800010000040000000000000002400000000020000080000000020000000000000000000000000200000000010000000000000000003CFE20
:5CDD0400000000000000000000000000000000000000000000000000000000000000000000000000000000000000000000000000000000000000000000000000000000000000000000000000000000000000000000000000000000000000DCFFE8
:5CDD6000000000000000000000000000000000000000000000000000000000000000000000000000000000000000000000000000000000000000000000000000000000000000000000000000000000000000000000000000000000000000DCFF8C
:5CDDBC00000000000000000000000000000000000000000000000000000000000000000000000000000000000000000000000000000000000000000000000000000000000000000000000000000000000000000000000000000000000000DCFF30
:5CDE1800000000000000000000000000000000000000000000000000000000000000000000000000000000000000000000000000000000000000000000000000000000000000000000000000000000000000000000000000000000000000DCFFD3
:5CDE7400000000000000000000000000004010000000000000000010000000000000000000000000000000000000000000000000000000000002000000080000000000000000280000000000000000000000000000000000000000000000D8FFE9
:5CDED00000080200000000000000000000001000000000000000000000000000000000000000001000000000000000000000000000000000000000000000010000000000000000000000000000000000000000000000000000000000000074FE59
:5CDF2C00000000000000000000000000000000000000000000000000000000000000000000000000000000000000000000000000000000000000000000000000000000000000000000000000000000000000000000000000000000000000DCFFBE
:5CDF8800000000000000000000000000000000000000000000000000000000000000000000000000000000000000000000000000000000000000000000000000000000000000000000000000000000000000000000000000000000000000DCFF62
:5CDFE400000000000000000000000000000000000000000000000000000000000000000000000000000000000000000000000000000000000000000000000000000000000000000000000000000000000000000000000000000000000000DCFF06
:5CE04000000000000000000000000000000000000000000000000000000000000000000000000000000000000000000000000000000000000000000000000000000000000000000000000000000000000000000000000000000000000000DCFFA9
:5CE09C00000001000000000000000000000020000000000000000000000000000000000000000000000000000000000000000000000000000010000000000000000000000000000000000000000000000000000000000000000000000000CCFC2F
:5CE0F800000000000000000000000000000000000000000000000000000000000000000000000000000000000000000000000000000000000000000000000000000000000000000000000000000000000000000000000000000000000000DCFFF1
:5CE15400000000000000000000000000000000000000000000000000000000000000000000000000000000000000000000000000000000000000000000000000000000000000000000000000000000000000000000000000000000000000DCFF94
:5CE1B000000000000000000000000000000000000000000000000000000000000000000000000000000000000000000000000000000000000000000000000000000000000000000000000000000000000000000000000000000000000000DCFF38
:5CE20C0000400000000000000000201000800000000040000000800000000000000000000000000100000000000000000000000000000000000000000000000000000000000000000000000000000000000000100000000000020000080030FFBC
:5CE26800000000000000000000000000000000000000000000000000000000000000000000000000000000000000000000000000000000000000000000000000000000000000000000000000000000000000000000000000000000000000DCFF7F
:5CE2C4000080000000000000000010200040000000002000000000010000000000000000000080000000000000000000000000000000000000000000000000000000000000000000000000000000000000000020000000000001000004009CFFAD
:5CE3200000000000000000000000A01000000410000000000800800000000000000000000000000000000000000000000000000000000000000000000000000000000000000000008000000002000000000000020000000000100100000084FD3F
:5CE37C000000000000000000000020100000001000000000080080000000000000000000000000000000000000000000000000000000000000000000000000000000000000000000800000000200000000000000000000000000040000008CFE6D
:5CE3D800000000000000000000000000000000000000000000000000000000000000000000000000000000000000000000000000000000000000000000000000000000000000000000000000000000000000000000000000000000000000DCFF0E
:5CE43400000000000000000000000000000000000000000000000000000000000000000000000000000000000000000000000000000000000000000000000000000000000000000000000000000000000000000000000000000000000000DCFFB1
:5CE4900010000000000000000000000000000000000000000000000000000000000000000000000000000000000000000000000000000000000000000000000000000000000000000000000000000000000000000000000000040000000088FF95
:5CE4EC00000020000000000000000000000000000000000000000000000000000000000000000000000000001000000000000000000000000000000000000000000000000000000000000000000000000000000000000000000000000000CCFCDC
:5CE54800000000000000000000000000000000000000000000000000000000000000000000000000000000000000000000000000000000000000000000000000000000000000000000000000000000000000000000000000000000000000DCFF9C
:5CE5A400000000000000000000000000000000000000000000000000000000000000000000000000000000000000000000000000000000000000000000000000000000000000000000000000000000000000000000000000000000000000DCFF40
:5CE60000000000000000000000000000000000000000000000000000000000000000000000000000000000000000000000000000000000000000000000000000000000000000000000000000000000000000000000000000000000000000DCFFE3
:5CE65C00000000000000000000000000000000000000000000000000000000000000000000000000000000000000000000000000000000000000000000000000000000000000000000000000000000000000000000000000000000000000DCFF87
:5CE6B800000000000000000000000000000000000000000000000000000000000000000000000000000000000000000000000000000000000000000000000000000000000000000000000000000000000000000000000000000000000000DCFF2B
:5CE71400000000000000000000000000000000000000000000000000000000000000000000000000000000000000000000000000000000000000000000000000000000000000000000000000000000000000000000000000000000000000DCFFCE
:5CE77000201000000000000000000000000000000000000000000000000000000000000000000002000000000000000000000000000000000000000000000000000000000000000000000000000000000000000000000000000000000000CCFE51
:5CE7CC00000000000000000000000000000000000000000000000000000000000000000000000000000000000000000000000000000000000000000000000000000000000000000000000000000000000000000000000000000000000000DCFF16
:5CE82800000000000000000000000000000000000000000000000000000000000000000000000000000000000000000000000000000000000000000000000000000000000000000000000000000000000000000000000000000000000000DCFFB9
:5CE8840000000000000000000000000000000000000000000000000000080000000002000000000000000000000000000000000000000000000000000000000000000000000000000000000000000000000000000000000000000000000074FDBD
:5CE8E000000000000000000000000000000000000000000000000000000000000000000000000000000000000000000000000000000000000000000000000000000000000000000000000000000000000000000000000000000000000000DCFF01
:5CE93C0000000040000000000000000000004002080000002000000000020000000000000000000000000000000000000000000000000000100000000000010000310000000000000000000000000000000000000000000000000000200610FD5E
:5CE99800000000000000000000000000200000000000000000000000008000000008000000000408000000000000000000000000000000000000000000000000000000000004000004008000000A000000000000008008000000000040003CFDDC
:5CE9F40000000000000000000000000000040000000000000000000000000000000000000000000000000000000000000000002000000000000000000000000000000000000000000000000000000000000000000000000400008000000050FDD2
:5CEA5000000000000000000000000000000000008000000000100000000000000000010000000000000000000000000000000000000000000000000000000000000000000000100000000000000000000000000000000000000000000000C4FE07
:5CEAAC000000000000000000000000000000000000000000000000000000000000000000000000000000000000000000000000000000000000000000000000000000000000080000000000000000000000000000000000000000000000005CFFAB
:5CEB080000000000000000000000000000000000000000000000000000040000000000000000000000000000000000000000000000000000000000000000000000000000000000000000000000000000000000000000000000000000000098FF16
:5CEB640040000000000000000000000000000000000000000000000000000080000000000000000000000000800000000000000000000000000002000000000000000000000010000000000000002000002000000000000000000000000024FDA2
:5CEBC00000000000000000000000000000000000000000000002C00000020200000000000000000000000080000000000000000000000000000000000000020000000000000000000000000000000000000200000000000000000000004034FD3E
:5CEC1C00160000000000000000000000000000000000000000000000000000000000000000000000000000000000000000000000000000000000000000000000000000000000000000000000000000000000000000000000000000000000E8FDA1
:5CEC780000000000000000000000000000000000000000000000000000000000000000000000020000000000000000000000000000000000000000100000000000000000000000000000000000000000000000000000000000000000004088FC6A
:5CECD40080000000000000000000001004000010000000000000810000000000100002100010000000000000000000000000000000000000080000000000800000000000802000008040100800010000000120100000001008000000001088FEAD
:5CED30000000000000000000000000000000000000000000000000000000000004000000000000000000000000100000000000000000400020000000000000000000080000000001000000000000000000000000000000000000000000007CFD91
:5CED8C00400000000000000000000020020000080002000000800021000000000C000120200400000000000000040000000000000080420018000000000000010000020000110001408008100002000080001020000000081002000000080CFE24
:5CEDE80000051008000000000000000281025090000000000800902001010050808000402408040060000000008000000000000000800000200004000020000000204080040010008150100A2240000000A820010400011004002000080068FE7E
:5CEE44000000100800000000000000000002401000000000080080200000004000000020200804000800000000000000000000000000000020000400000000000080000000001000804010080240000000802000020000100000000008006CFEDA
:5CEEA000800000000000000000000000000000000000000000000000000000000000000000000000100000000000000000000000000000000000000000100000000000000000000001000000000000000000000000800000100000000000DCFF0A
:5CEEFC00000000200000000000000040000800012000000000100002000008000100000000001000020000000001000000000000000000000040000000000000008000000002400000000120000400000000024000000001200000000010ECFE7F
:5CEF5800080200000000000000000000000000000000000000000000000000000000000000000000000000000000000000000000000000000000000000000000000000000000000000000000000000000000000000000000000000000000E7FE6E
:5CEFB40000000400000000000000000000008000000000000000000000000000000000100000000000000000000000000000000000000000000000000024040000000000000000000000000000000000000000000000000000000000000064FEE3
:5CF01000000000000000000000000000000000000000000000000000000901000000200000808000000000000000000000000000000000000012000000201000000000000000000000000000200000000000000000004000000000000000D8FE02
:5CF06C00000000000000000000000000000000000000000000000000000000000000000000000000000000000000000000000000000000000000000000000000000000000000000000000000000000000000000000000000000000000000DCFF6D
:5CF0C800000000000000000000000000000000000000000000000000000000000000000000000000000000000000000000000000000000000000000000000000000000000000000000000000000000000000000000000000000000000000DCFF11
:5CF12400000000000000000000000000000000000000000000000000000000000000000000000000000000000000000000000000000000000000000000000000000000000000000000000000000000000000000000000000000000000000DCFFB4
:5CF18000000000000000000000000000000000000000000000000000000000000000000000000000000000000000000000000000000000000000000000000000000000000000000000000000000000000000000000000000000000000000DCFF58
:5CF1DC0000000000000000000000001000000000000000000000000000400000000000000000008000000000000000000000000000000000000000000000000000000000000000000002000000000000400204020000000000000000800058FEE7
:5CF23800000000000000000000000000000000000000008000000000000000000000000000000000030000000000000000000000000000000000000000800800000000000000000000000000000000000040000000000000000000000200A8FE87
:5CF29400008002000000000000000000400000000000000000200000000014000000000000002800050000000002000000000000000000000080000000004000000001000000800000000000000800000000000000000002000000000020FCFF93
:5CF2F00000000400000000000000000004A00000000000000000000000000000000000000000000000000000000000000000000000000000200004000010000000000000002000000000000000000000400100000000000000000000000090FDF8
:5CF34C00200000000010000000000000000008008000000002000000000000000000000000000000000000200000000000000010000000000002400000000046000000000000000000080000000000004000000000000804000000008000FCFF24
:5CF3A8000000000000000000000000000000000200000000000000000000000000000000000000000000000000000000000000000000000000800010000000000800000000000000000002000000000000000000000000020000000000204CFC03
:5CF4040060800000003000000000000000600000800102000600000000000000000000000000000000000060000000000000003000000000180003000000800701000000000000006000000000000000C00000000060000C000000000600C4FC2E
:5CF46000A01100000010000000000000002000008046000002000000000000000000000000000000000000200000000000000010000000000800010000008026000000000000000020000000000000004000000000200004000000000200F4FE50
:5CF4BC000044000000C00800000000000080050000200000180100000000000000000000000000000000008005000000000000C00400000060028C0200000016000000000000000080090000000000000003000000804530060000005800ACFD53
:5CF51800C001000000E020000000000000C04100000701001C040000000000000000000000000000000000C041000000000000E02000000070100E00000000070100000000000000C0810000000000008003040000C00138000000001C20A0FE7B
:5CF574008001000000C00000000000000080010000060100180000000000000000000000000000000000008001000000000000C00000000060000C0000000006000000000000000080010000000000000003000000800130000000001800CCFF8F
:5CF5D0008051000000C00000000000000080010000160000180000000000000000000000000000000000008001000000000000C00000000060000C00000000460100000000000000800100000000000000030000008001300000000018009CFFC3
:5CF62C0004080000001000000000600400200000800000000200000000010000000046000000000000000000080000000000000004000000080040000000002010000000000000400008008000000000001000000020000400000000028060FCBB
:5CF68800000002000000000000000080000000000000000000000000000000000000000800000000000000000002000000000000000100000000001000000000080000000000000010000200000000000000040000000000000000000000C0FCAF
:5CF6E40068000000003000000000788000600000800102000600000000030000008007010000000000000060000000000000003000000000180003000000800130000000000000036000008001020000C00000000060000C10000000060095FEAF
:5CF7400020000000001000000000680400200000804600000200000000010000008006000000000000000020000000000000001000000000080001000000800010000000000000012000008046000000400000000020003402000000020098FF83
:5CF79C008411010000C0000100006001008005000000010018050000008C080000002600000000000000008005000000000000C00000000060012C0200000006C08800000000008C820100000000000000030000008009020A000000188500FD99
:5CF7F800C001000000E000000000701000C04100000700001C000000000E00000000070100000000000000C041000000000000E02000000070200E0000000007E80000000000000EC0010100070400008083000000C00138000000001C0010FDCC
:5CF854008801000000C0000000006000008001000006000018000000000C000000000601000000000000008001000000000000C00000000060000C0000000006C00000000000000C8001000006000000000300000080013000000000180021FC0E
:5CF8B0008001000000C0000000006014008001000026010018000000000C000000001600000000000000008001000000000000C00000000060000C0000000006C00000000000000C800100000604000000030000008001302200000018003CFC35
:5CF90C0084210000001000000000000200200000012000008000000000000000000000000002000000000020000000000000001000004000000240000004002010000000000002018011008000000000002300000000080000001000188158FD02
:5CF968000000000000000000000000800000000040000800002000000000000000000000000000000000000000000000000000000000000000800010000000000800000000008000000002000000000000000400000000020000000000204CFED1
:5CF9C400E801000000300000000018000060000C80010000060000000000000000000000000600000000006000000000000000300000C00018000300000C90013000000000180003E041008001020000C003000000600000000030001E00FDFF59
:5CFA2000A005010000100000000008000020000480000000020000000000000000000000000200000000002000000000000000100000400008000100003482001000000000080001A0090080460000004083000000200000000010009A04ECFFF1
:5CFA7C008441000000C00000000060120080513009160000180500000000000000000000001804000000008001010000000000C02000006360044C0200800826C08000000060004C8011000020010000008B0000008009000000C0085884F8FE6D
:5CFAD800C001000000E020000000700000C00138000702001C0000000000000000000000001C0000000000C001000000000000E00000800370100E0000380007E20000000070800EC8410000070000008003000000C041000000E0001D0084FE83
:5CFB34008801000000C00000000060000080013000060000180000000000000000000000001800000000008001000000000000C00000000360000C0000300006C00000000060000C804100000600000000030200008001000000C000180449FF62
:5CFB90008005020000C00000000060000080013000060000180000000000000000000000001800000000008001000000000000C00000000360000C0000300A06C00000000060000C8001000006010000000B0000008001000000C00018010CFF77
:5CFBEC002400000000C008000000000200000830024600008000000000000000000020000080001000000000080000000000001000000000080000000004002010000000000002408011000020000000400000000020000001000000028084FF72
:5CFC480000000000000000010000008000000002400008000020000000000000000000080000200004000000000200000000000000000000000000000000000008000000000080001000020000080000000000000000000040000000000094FDD4
:5CFCA4006880000000F04000000018000060003CC00700000600000000000000008001000006C0000000006000000000000000300000000018000000000C90013000000000180003E001018001000000C00001000060000C000000000600FDFC05
:5CFD0000A011000000D00000000008000020003481160100020000000000000000800000000240000000002000000000000000100000000008000000003482001000000000080001A011008000000000402300000020000400000000020098FE17
:5CFD5C000400020000C0280000006011008049B000460800180100000000000000000604001804230000008045000000000000C0020000006002000000001216C00200000060010C820100001602000000080000008045B0000000005880A4FCF3
:5CFDB800C001000000E000000000700000C00138080700001C0400000000000000000700001C8003010000C001000000000000E0200000007020000000380007E22000000070400EC0410000070000008083000000C00138100000001C1010FF70
:5CFE14008841000000C00000000060000080013008060000180000000000000000000600001800030000008001000000000000C0000000006000000000304006C00000000060000C800101000600000000830000008001300000000018008DFE0F
:5CFE70008011000000C0020100006000008001B000460200180000000000000000000600001800030000008001000000000000C0000000006000000000300106C00000000060000C8005000006000000002300000080013000000000180044FD14
:5CFECC00200000000000040000000800002000048000000080400000000000000080000000024000000000000800000000000000040000000800010000000120000400000000028C20000000460000004000000001000800010000008080E4FE2E
:5CFF2800000000000000000100000000000000000000000000200000000000000000000000000000000000000002000000000000000100000000000000004000080001000000800010000000000800000000000000000002400000000020A8FC72
:5CFF84006080000000300000000018000060000C8001000006C0000000000000008001000006C0000000006000000000000000300000000018200300000C8001300000000018000F6080008007000000C00000000360000C0000000006001DFF98
:20FFE000FFFFFFFFFFFFFFFFFFFFFFFFFFFFFFFFFFFFFFFFFFFFFFFFFFFFFFFFFFFFFFFF21
:020000040001F9
:5C000000A81100000010000000000800002000048000000002400000000000000080000000024000000000200000000000000010000000006804010000048000100000000008000DA211008026080000400000000120000400000000020058FEC7
:5C005C000004000000C00800000060040080053022000400180013040000000000000600005800880000008005000000000000C02000000000808C1000302006C40400000060140C1008000016000000001000000C8011B00800000018852CFCB1
:5C00B800C041000000E020000000704000C0013A000100001C8403000000000000000708001C8400000000C001020000000000E00000000070000E0000380007E02000000070000EC041000007020000800002000EC84138000000001C00FCFC20
:5C0114008401020000C00000000060000080013000060200180003000000000000000600001800030100008001000000000000C00000000060000C0000300006C00000000060000C8241000006040000000301000C80013000000000180069FED6
:5C0170008001000000C00000000060000080013000460000180003000000000000000600001800230000008001000000000000C00000000060200C0000300006C00000000060002C8005000026000000002300000C80013000000000180018FD38
:5C01CC00842100800000040000000800000008008100000002000000020000000000200000800023000000200004000000000000040000006004010000300246C0080000006004402000000046000000001000000020000400001000800068FE55
:5C0228000000000000000001000000000000000240000000000000008000000000000008000020000400000000000000000000000001000000800000000040000800010000008000100000000008000000000400000000000000000000204CFCBD
:5C028400E801008001300000000018000060000C800102000600001800000000008001000006C08300000060000C0000000000300000000078100300003C8807F0000100007800036000008007000000C00000000060000C00003000060000FDF1
:5C02E000A00101800010000000000800002000048046000002000008000000000080000000024013000000200004000000000010000000006800010000348206D10800000068110120000080460100004000000000200004000010000200C5FEF3
:5C033C008411000026C0020000006000008051300A200000180000600000000000002601005800130000008005300200000000C00400000060008C0200300A46C12000000060122C000400001600000000030000008011304200C048180304FEA6
:5C039800C041000007E820000000704000C00138000704001C0400704000000000000700001C8483000000C081381000000000E02000000070100E0000380007E00000000070000E42400000070400008003020000C041380000E0001C0098FCBC
:5C03F4008841000006C00000000060000080013000060100180000600000000000000600001800830000008001300000000000C00000000060000C0000300006C12000000060000C808100000601000000030000008001300000C0001880F8FE83
:5C0450008001000006C00000000060000080013000460000180000600000000000000600001800030000008001300000000000C00000000060110C0000302246C00800000060140C801100002600000000030000008001300000C0001800C8FC44
:5C04AC0004080080000004000000080000200004800000000200000000000000000020000080001000000080110000000000000004000000000201000000012000040200000800010008008000000002400008000080113002000000028024FE05
:5C05080000000200000000010000000000000000000000000000000000000000000000080000200004000000000200000000000000010000008000000000400008000100000000000000020000000000000000000000000240000000000084FFD5
:5C0564006800008001300000000018000060000C800102000600000000000000008001000006C000000000E001000000000000300000000018000300000C800130000600001800036000008001020006C000190000E0013C08000000060061FE78
:5C05C000200000800010000000000800002000048046000002000000000000000080000000024000000000A05100000000000010000000000800010000048000100002000008000120000080460000024023080000A049340200000002005CFD03
:5C061C008409020006C40000000060110080493041200400581000000000000000001600009804130000008011000000000000C00200000060204C0200302206C80218000060082C84110200100100180110628000800931010000009880F8FFC1
:5C067800C001000007E020000000700000C00138000700001C0000000000000000000702001C8003020000C041000000000000E02000000070000E0000380007E0201C200070000EC00100000700001C9003700000C00138080000001C048CFE1E
:5C06D4008801000006C00000000060000080013000060000180000000000000000000600001800030000008041000000000000C00000000060000C0000300006C00018000060000C8001000006000018000360000080013008000000180031FCC4
:5C0730008001000006C00000000060000080013000060100180000000000000000000600001800030000008011000000000000C00000000060000C0000300006C00018000060000C800100001601001800A3600000800131010000001800BCFF65
:5C078C000408048000C00800000008000100080400460000800000000000000000800010000200100002002000000000000000100000000008000120000400200004000000080001000804002010000040000000002000008100100080806EFC19
:5C07E80000000200000000010000000000000002000008000020000000000000000000000000000004800000000000000000000000000000000000000000000008000100000000000000020000080000000000000000000040000000002028FC6D
:5C08440068000C8001F04000000018000364000C900700000600000000000000008001300006C0001800006000000000000000300000000018200360800C9001300000000018000360000C8001300000C00000000060000C800130000600A5FF45
:5C08A0002000048000D00800000008008D200034821604000200000000000000008000100002400008000020000000000000001000000000680401A011348200100000000008000120000480001000004000000000200004800010000280E9FEF1
:5C08FC008411301046C822000000601280811100011604005804000000000000000026C1025900236480008045000000000000C00400000000112C0208802046C00800000060140C8809324126C0020000030000008009300006C0429800B9FC5C
:5C095800C0013A0007E00000000070000EC04138080700001C00000000000000000007E0001C8803700000C001000000000000E04000000070000EC0013A0007E42000000070000EC001380007E440008083000000C041380807E4001C0408FF24
:5C09B4008801300006C08000000060000C800130000600001800000000000000000006C0001800036000008001000000000000C00000000060100C8001300006C00000000060000C8001300006C0000000030000008001300006C000188010FF34
:5C0A10008001300006C00400000060000C840130222608001800000000000000000006C0001800036000008001000000000000C00000000060040C8001B10806C00000000060000C8001300006C0000000030000008001300006C000180020FD02
:5C0A6C0014000000000000000000000000000000000000000000000000000000000000000000000000000000000000000000000000000000000000000000000000000000000000000000000000000000000000000000000000000000008062FD3B
:5C0AC800200004800010000240000800012000048000100002400008000120000480001000024000080001200004000000000010000240000800012000048000100002400008000120000480001000024000080001200004800010000200BCFCEA
:5C0B2400080000000000000000000000000000000000000000000000000000000000000000000000000000000000000000000000000000000000000000000000000000000000000000000000000000000000000000000000000000000000C5FEAA
:5C0B80002C000480001000024000080001200004800010000240000800012000048000100002400008000120000400000000001000024000080001200004800010000240000800012000048000100002400008000120000480001000028029FD37
:5C0BDC000801200004800000000040000800012000040000100002400008000000000480001000024000000001200000000000800000000240000800012000048000100000400008000120000480001000024000080001200004800010004DFF8B
:5C0C38000000000000000002400000000000000000001000000000000000200004000000000000000000010000000000000000000002000000000000000000000000004000000000000000000000000000000000000000000000000000009CFD0E
:5C0C940084001000024000000000200004800010000200000800012000040000000002400008000120000080001000000000004000000001200004800010000240000800002000048000100002400008000120000480001000024000088094FF01
:5C0CF0000000000000000002400000000000000000001000000000000000200004000000000000000000010000000000000000000002000000000000000000000000004000000000000000000000000000000000000000000000000000009CFD56
:5C0D4C00000000000000000000000000000000000000000000000000000000000000000000000000000000000000000000000000000000000000000000000000000000000000000000000000000000000000000000000000000000000000DCFF70
:5C0DA800000000000000000000000000000000000000000000000000000000000000000000000000000000000000000000000000000000000000000000000000000000000000000000000000000000000000000000000000000000000000DCFF14
:5C0E0400000000000000000000000000000000000000000000000000000000000000000000000000000000000000000000000000000000000000000000000000000000000000000000000000000000000000000000000000000000000000DCFFB7
:5C0E60000000000000000000000000000000000000000000000000000000000000000000000000800000000000000000000000000000000000000000000000000000000000000000000000000000000000000000000000000800000000005CFF53
:5C0EBC00000000000000000000000000000000000000000000000000000000000000000000000000000000000000000000000000000000000000000000000000000000000000000002000000000000000000000000000000000000000000FCFFDD
:5C0F180000100000000000000000002000000000000000000000000000000000000000000000000000000000000000000000000000000000000000000000000000400000000000000000000000080000001000000000000000000000000040FDB8
:5C0F7400000000000000000000000000000000000000000000000000000000000000000000000000000000000000000000000000000000000000000000000000000000000000000000000000000000000000000000000000000000000000DCFF46
:5C0FD000000000000000000000000000000000000000000000000000000000000000000000000000000000000000000000000000000000000000000000000000000000000000000000000000000000000000000000000000000000000000DCFFEA
:5C102C00000000000000000000000000000000000000000000000000000000000000000000000000000000000000000000000000000000000000000000000000000000000000000000000000000000000000000000000000000000000000DCFF8D
:5C108800000000000000000000000000000000000000000000000000000000000000000000000000000000000000000000000000000000000000000000000000000000000000000000000000000000000000000000000000000000000000DCFF31
:5C10E4000000000000000000000000000000000000000000800000000000000000000000000000000000000000000000000000000000000000000000000000000000000000000000000800000000000000000000000000000000000000005CFFCD
:5C1140000000000000000000000000000000000000200000000000000000000000000000000000000000000000000000000000000000000000000002000000000000000000000000004000100000000000000000000000000000000000009CFE47
:5C119C00000000000000000000000000000000000000000000000000000000000000000000000000000000000000000000000000000000000000000000000000000000000000000000000000000000000000000000000000000000000000DCFF1C
:5C11F800000000000000000000000000000000000000000000000000000000000000000000000000000000000000000000000000000000000000000000000000000000000000000000000000000000000000000000000000000000000000DCFFC0
:5C125400004000000000000000000000000240000000000000000000000000000000000000000000000000004000000000000000000004000000000200000000010000000000000000000000000000000000000000800000000000000800C0FE2F
:5C12B000000000000000000000000000000000000000000000000000000000000000000000000000000000000000000000000000000000000000000000000000000000000000000000000000000000000000010000000000000000000000CCFE17
:5C130C00008000000000000000000000000480000000000000000000000000000000000000000000000000008000000000000000000008000000000400000000020000000000000000000000000000000000020000400000050000000400C4FEE6
:5C13680000000000004000000080000040800000000000000800A00044000200000000010008000000000000000000000000000000800000004400025000000000000000000000040000100000000000000020000080000020000088000910FE29
:5C13C40000000000004000000000010000800000000000000800800000000800000000010008000000000000000000000000000000000000000000024000000000000000000000040000080000000000000010000020000000000000000028FDD0
:5C142000000000000000000000000000000000000000000000000000000000000000000000000000000000000000000000000000000000000000000000000000000000000000000000000000000000000000000000000000000000000000DCFF95
:5C147C00000000000000000000000000000000000000000000000000000000000000000000000000000000000000000000000000000000000000000000000000000000000000000000000000000000000000000000000000000000000000DCFF39
:5C14D800000000000000000000000000000000000000000000000000000000000000000000000000000000000000000000000000000000000000000000000000000000000000000000000000000000000000000000000000000000000000DCFFDD
:5C153400004000000000000000000000000000000210000000000000000000000000000000000000000000000000000000000000000000008010000000000000000000000000000000000000100000000000000000002000000000000000E0FF6A
:5C159000000000000001000000000000000000000000000000000000000000000000000000000000000000000000000000000000000000000000000000000000000000000000000000000000000000000000000000000000000000000000CCFF33
:5C15EC00000000000000000000000000000000000000000000000000000000000000000000000000000000000000000000000000000000000000000000000000000000000000000000000000000000000000000000000000000000000000DCFFC8
:5C164800000000000000000000000000000000000000000000000000000000000000000000000000000000000000000000000000000000000000000000000000000000000000000000000000000000000000000000000000000000000000DCFF6B
:5C16A400000000000000000000000000000000000000000000000000000000000000000000000000000000000000000000000000000000000000000000000000000000000000000000000000000000000000000000000000000000000000DCFF0F
:5C170000000000000000000000000000000000000000000000000000000000000000000000000000000000000000000000000000000000000000000000000000000000000000000000000000000000000000000000000000000000000000DCFFB2
:5C175C00000000000000200000000000000000000004000000000000000000000000000000000000001000000000000000000000000000000000000000000000000000000000000000000000000000000000000000000000000000000000ACFE53
:5C17B80000000000000080000000000000000000004000000000000000000000000000000000000000000000000000000000000000000000000000000000000000000000000000000000000000000000000000000000000000000000000018FFFE
:5C181400000000000000000000000000000000000000000000000000000000000000000000000000000000000000000000000000000000000000000000000000000000000000000000000000000000000000000000000000000000000000DCFF9D
:5C187000000000000000000000000000000000000000000000000000000000000000000000000000000000000000000000000000000000000000000000000000000000000000000000000000000000000000000000000000000000000000DCFF41
:5C18CC0000000800100000000000000000000000000000000000000000000000000000000000002000000000000000000000000000000000000000000001000000000000000000000000000000000000000000000000000400000000004058FDEE
:5C192800000000000000000000000000000000000000000000000000000000000000000000000000000000000000000000000000000000000000000000000000000000000000000000000000000000000000000000000000000000000000DCFF88
:5C198400020002000000000000000008000000000800000000000000000000000000000000000004000000000040000000000080000000000000000000000090010200000000008400010000420000000210001000000000000000000200ECFCC9
:5C19E000000400000000000000000008000000800000010000000000080000000000000000000000000000000000000000000000000000000000000000000000000000000000000000800000000000000040000000008800008000000000CCFE84
:5C1A3C00000000000004000000000000000000000000000000000000000000000000000040000000000000000000000000000000000040000000000000000000000000000000000000000000000000000000000000000000000040000100D8FEB3
:5C1A980000000000000000000000000000000000000000000000000100200000000000080000000000000000000000000000000000000000000000000000000000000000000000000000000000000000000000000000000000002000000064FF46
:5C1AF40000000000000000000000000010000000000000000000000000000000000000000000000000000000000000000000000000000000000000000000000000000000000000000000000000000000000000000000000000000000008044FFC3
:5C1B5000000000000000000000000000000000000000000000000000000000000000000000000000000000000000000000000000000000000000000000000000080000200000000000000000000000000000000000000000000000000000F4FF1E
:5C1BAC00000000000000000000000000000000000040000000000000000000000000100000000000000000000400000000000000000000000000000000000000000000000000000000000000000000000020000000000000000000000000CCFDA0
:5C1C080000C001000040000000000000000000001004000000000000000000000000000000100000000000000000000000000000000000004000000000000004000000000000800000080000C00000000000040000000000000000000000CCFE01
:5C1C64001C00000000000000000000000000000000000000000000000000000000000000000000000000000000000000000000000000000000000000000000000000000000000000000000000000000000000000000000000000000000C03FFC0D
:5C1CC0000000000000000000000000000000000000000000000000000000000000000000000000000000000000000000000000000000000000000000000000000000000000000000000000000000000000000000000000000000000000C010FFF9
:5C1D1C0000000000000100000000200000000010880000000004000000000200000000400000000000000000001000000000004000000400000000008000000200000800001000000040000000400000000120000400400000000000000040FD5C
:5C1D7800000000000040000000000000000000000002100000000000000000000000000000040400000000000000000000000000000040000000000000000000000000000000000102000000020000000000000000000000000000000000ACFCC8
:5C1DD400000000001412140000001000000000089001100000085000000004000000002000021000000000000008000000000020000048000000000080000001000004000010000108800080002000508000500102008000000000008002CCFE15
:5C1E30000000040820800600008120000400008401000000080000200040000000000080028004A02000008030800A000000000000A800001000048040000A10402000050500100080401000000002480088004534800200A40210008800B4FC77
:5C1E8C0000000004000000000002210004000000000000000800001000000000000000000000048020000040000008000000000000080000000004808000080020200004010010002000110000000002000002000480000000020000080030FC73
:5C1EE80000000000004000000000000000000000000000000000000000000000000000400000000000000000400000000000000000000000000000000000000000000000000000000000000000000000000000000000000010000000000088FF47
:5C1F4400000001000000800000000040000000012000040000100000400000000000000400001000024000000001000000000000800000000040000800002000048000000000400008000100000400000000020000000001200000000010F8FFD1
:5C1FA0001C0000000000000000000000000000000000000000000000000000000000000000000000000000000000000000000000000000000000000000000000000000000000000000000000000000000000000000000000000000000000D1FEFA
:5C1FFC00002000000000020000000000000000000020000000000000000000000000000000000000000000000000000000000000000000005000000000800204000000000000002000000000800000000000000000000000000000000000A8FC2D
:5C205800000000000020000000000000000000010000080000000000000000000000000000000000000000000001000000000000000000000000000000080000000000000000000000200000040000000000000000010000000000000010E8FCE1
:5C20B400000000000000000000000000010000000000000000000000000000000000000000000000000000000000000000000000000000000000000000000000000000000000000000000000000000000000000000000000000000000000CCFE05
:5C2110000000000000000000000000000000000000000000000000000000000000000000000000000000000000000000000000000000000000000000000000000000000000080000000000000000000000000000000000000000000000005CFF10
:5C216C0000000000000000000000000000000000000000000000000000000000000000000000000000000000000000000000000000000000000000000000080000000000000000000000000000000000000000000000000000000000000054FFBC
:5C21C800000000000000000000000000000000000000000000000000000000000000000000000000000000000000000000000000000000000000000000000000000000000000000000000000008000000000000000000020000000000000D4FD4A
:5C222400000000000000000000000000000000000000000000000000000000000000000000000000000000000000000000000000000000000000000000000100000000000000000000000000000000000000000000000000000000000000DCFE83
:5C2280000000000000000000000000000000000000000000000000000000000000000400000000000000000001000000000000000000000000000000008000000002000000000400000000000000000000000000000000000000000000014CFC2E
:5C22DC000000000000000001000000800000000040000800000000000000000000000008000000000400000000020000000000000000000000800000200040000800010000008000100002000008000000000400000000024200000000202CFFB9
:5C233800A00000000000000000000000040000100002000000000000000000000000000000000001000000000000000000000000000000002000008000100000000000000000000080000000020000000001000000000010000000000000D8FE79
:5C2394000000000020000000000000000000000001000000000000000000000804002000000000000000010000040000000000000000001000000000000000200000000010000040000800800000000000000800000000040000000000000CFF7C
:5C23F00000000000000800000000000000000000400000000000000000000000020000080000000000000000000000000000000000000000040000000000000008000000000400001000020000004000000000000000000000000000000098FE47
:5C244C000000008001000000000000000000000C0000000000000000000060000C8001000000000000000300000C0000000000000000C0000000000000008001000000C0000000036000008001300000000018000000000C00000000000090FEE4
:5C24A80000000080000000000000000000000004000000000000000000002000048000000000000000000100000400000000000000004000000000000000800000000040000000012000008000100000000008000000000400000000000018FFD7
:5C250400000000004601000000000000000000300A0000000000000000008031304206040000000000004C0000B00000000000000000000B00000000000000C6000000002304008C8049000026C0000000006004000000B0000000000000E0FEAC
:5C2560000000000007000000000000000000003800000000000000000000C001380007000000000000000E020038080000000000000080830000000000000007000000800300000EC401000007E200010000701000000038200000000000E8FF87
:5C25BC0000000000060000000000000000000030000000000000000000008001300006000000000000000C000030000000000000000000030000000000000006000000000300000C8001000006C000000000600000000030000000000000A8FE05
:5C26180000000000060000000000000000000030000000000000000000008001300006000000000000000C000030000000000000000000030000000000000006000000000300000C8001000006C000000000600000000030000000000000A8FEA8
:5C267400040004002000000000000002000000000100C00800000000000080110001200000000000080001000004000000000000000000100000000000040046000000400000008C0008040000100000000008000020000001000000008068FD08
:5C26D00000000000000800000000008000000000400000000100000000000000024000080000000000000000000000000000000000000000040000000000000008000000000000001000020000000000000000000000000040000000000000FE3F
:5C272C0008000C8001000000000018000000000C0000F020000000000000E0010C8001000000000018000300000C0000000000000000C00000000000000C8007000000C00000000F70000C0000300000000018000060000C00000000000015FD8F
:5C278800000004800000000000000800000000040000D004000000000000A0450480000000000000080001000004000000000000000040000000000000048026010000400000008D20000400001000000000080000200004000000000000CCFD3A
:5C27E400040030411601000000006002000000300200C0080000000000008049300016000000000060020C000030000000000000000000A30000000000300116040000000B02004C8801310200C008000000608400800130000000000080C0FE66
:5C284000000038000700000000007010000000381000E040000000000000C001380807020000000070100E020038080000000000000080030000000000381007000000800300000EC001381000E080000000700000C001390800000000005CFFA2
:5C289C00080030000600000000006000000000300000C0200000000000008001300006000000000060000C000030000000000000000000030000000000300006040000000300000C8201300000C00000000060000080013000000000000095FC7E
:5C28F800000030000600000000006000000000300000C0020000000000008049300006000000000060000C000030000000000000000000030000000000300026000000000300008C8001300000C000000000600000800130000000000000C8FF30
:5C29540004000400000000000000080000000004000000000000000000000008040020000000000008004000000400000000000000004000000000000000810000000000100000400008000100100000000000020000080001000000008034FDB5
:5C29B0000000000000000000000000000000000000000000000000000000000002000008000000000000001000000000000000000000000000000000000040000000000000040000100002400000000000000080000000024000000000002CFE2F
:5C2A0C0008000C4000000000000018000000000C4000000000000000000060000CC001000000000018000300000C0000000000000000C00000000000000C8001080000C00000000360000C0000300000000018000060000C00000000000079FEB3
:5C2A68000000B4000000000000000800000000B4000000000000000000002000B480000000000000080001000004000000000000000040000000000000048016000000400000000120000400001000000000080000200004000000000000D0FEF8
:5C2AC40004000042000000000000600000000000090000000000000000008005002206010000000060010C020030200000000000000000630000000000B00800020000002300008C8811300100C0040000006004008009B0200000000080E8FE1D
:5C2B20000000380000000000000070200000003800000000000000000000C001390007000000000070800E000038000000000000000080030000000000380007000000808300000EC001390800E020000000701000C0013900000000000054FC83
:5C2B7C0008003000000000000000600000000030000000000000000000008001300806000000000060000C000030000000000000000000030000000000300006010000000300000C8001300000C00000000060000080013000000000000085FD8D
:5C2BD8000000B0200000000000006000000000300A0000000000000000008001B00006000000000060000C000030000000000000000000030000000000300016000000000300000C8001300000C00000000060000080013000000000000024FE68
:5C2C3400040004000000000000000800000000040000000000400000000080110001200000000000080001000000010000000000000040000000000000308200000002001000000180110400001000000000000200000804000000000000BCFFC1
:5C2C90000000000000000000000000000000000000000000000000000000000002400008000000000000000000004000000000000000000000000000000040000000000000040000000002000000000000000080000000020000000000003CFF5B
:5C2CEC0008000C4000000000000018000000000C4000000000C000000000E0010C8001000000000018000300000C0000000000000000C00000000000003C8801080006E000000003E0010C0000300000000018000060000C00000000000014FF55
:5C2D48000000B4000000000000000800000000B400000000004000000000A001058000000000000008000100000400000000000000004000000000000034811600005A4000000001A049040000100000000008000020000400000000000025FD5B
:5C2DA400040000060000000000006000000000000000000000000B0000008051300126010000000060010C020030000000000000000000030200000000B00040000000219300000C8411302100C00800000060200080013210000000000088FF69
:5C2E00000000380000000000000070400000003820000000008003010000C001381007000000000070200E00003808000000000000008003000000000038080701001C800300000EC041380000E020000000700000C0013800000000000010FD9D
:5C2E5C0008003000000000000000600000000030200000000000030000008041300006000000000060000C000030000000000000000000030000000000300806000018040300000C8001300000C000000000600000800130000000000080E0FD51
:5C2EB8000000B008000000000000600000000030000000000000030000008005300006000000000060000C000030000000000000000000030000000000300016010058000300000C8045300000C00000000060000080013000000000000018FF8E
:5C2F14000000300220100000000000020000003082001000000000000000000830820000000000006004400000000100000000000000001000000000000480000000024000000040200000010000000000000002000008000100000000804CFCD2
:5C2F7000000000400008000000000080000000004000000000000000000000000240000000000000008000100000400000000000000000000400000000000000000000000000000010000040000040000000008000000002400000000000A0FCF9
:5C2FCC0000003C8801300000000018000000003C8001300000000000000060003C8801000000000078100300000C0000000000000000C00000000000000C8001000006E00000000360000C0000300000000018000060000C00000000000069FD37
:5C30280008003480001000000000080000000034A20010000000000000002000348000000000000068000100000400000000000000004000000000000004800000005A40000000012000040000100000000008000020000400000000000084FF0F
:5C3084000000301006C1080000006001000000300226C8000000000000008005320226040000000060844C000030020000000000000000130000000000304040000000006300004C8041300200C00800000060000080413006000000008004FF14
:5C30E0000000380007E0000100007010000000380807E040000000000000C001380807000000000070000E02003808000000000000008083000000000038000104001C880300000EC201380800E020000000704000C0013800000000000060FDC7
:5C313C000400300006C0000000006000000000300006C0000000000000008001300006000000000060100C000030000000000000000000030000000000300006080018000300000C8001300000C000000000600000800130000000000000A9FEF3
:5C3198000000301206C0000000006000000000B01006C0000000000000008001300A06000000000060010C000030000000000000000000030000000000300016000018050300000C8001300000C000000000600000800130000000000000B0FCEC
:5C31F400040004800000000000000800000000300200000400000000000100080400460000000000000240000004000000000000000000230000000000048000000002002300008C0008300200000000000060040080110001000000008024FCF8
:5C32500000000000000000000000000000000000400000000100000000000000020000080000000000800010000000000000000000000000040000000000000000000000000400001000024000004000000000800000000240000000000034FEB9
:5C32AC0008000CC001000000000018000000003C2000300000000000000360000C8007000000000018000300000C0000000000000000C00300000000000C8001080006E00300000F60003C00003000000000781000E0410C000000000000C5FF9B
:5C3308000000B480000000000000080000000034010010000000000000012000048016010000000008000100000400000000000000004093000000000004801600005A40A300002D22003421001000000000680400A01104000000000000F8FEAA
:5C336400040000014601000000006002000000300000C00000000000004C8001000916040000000060020C000030020000000000000000230000000000300120000080000300008C8241B00000C00400000060010080053001000000008080FD11
:5C33C000000038400700000000007010000000380800E04000000000000EC4010A0007000000000070100E02003808000000000000008083000000000038200702001C908300000EC001380800E020000000701000C04138080000000000FCFD42
:5C341C00080030000600000000006000000000302000C00000000000000C8001304006000000000060000C000030000000000000000000030000000000300006010018040300000C8001300800C0000000006000008001300000000000002DFCEF
:5C3478000000300A0600000000006000000000B00000C00000000000000C8001B00006010000000060000C000030000000000000000000030200000000300046000018008B00004C8201300200C000000000601400805130000000000000E4FFD1
:5C34D40004000080000000000000600400000004000000040000000000010008000146000000000000024000000001000000000000004000000001000000810000000240000000402000040000C008020000000200000830020000000080A4FE89
:5C353000000000100000000000000080000000000000000001000000000000000240000800000000008000100000400000000000000000000000000000004000000000000000000010000000000000010000008000000002400000000000BCFDC8
:5C358C0008000C8001000000000078800000000C0000300000000000000360000C8007000000000018000300000C0000000000000000C00000000300000C8001080006C00000000360000C0000F00006000018000060003C08000000000031FE8F
:5C35E80000000480000000000000680200000004000010000000000000012000048046010000000008000100000400000000000000004000000001000004801600000240000000012000040000D0240200000800002000340200000000005CFE9C
:5C364400040030020600000000006004000000300200C02400000000002C8201302106000000000060018C0000B00800000000000000001300002C0400300980000000102300000C9049300100C00418080060000080113002000000008044FDBC
:5C36A000000038080708000000007010000000381000E00000000000000EC001390007010000000070100E0200380000000000000000808300000E0000380007000004808300000EC001380800E0001D0000701000C0413808000000000060FD7E
:5C36FC00080030000600000000006020000000300000C00000000000000C8001300006000000000060000C0000300000000000000000000300000C0000300006000018200300000C8001300000C020180000600000800130000000000000E9FF37
:5C375800000030000600000000006000000000300000C00000000000000C8001300006040000000060000C0000300000000000000000000300000C0000300046010058000300000C8001300000C0041800006000008001B008000000000044FFD6
:5C37B400040004800000000200000800000000040000000480000000004020000480001000020000080001200000010000000000000040000000002000008100100002400008000120000400000000000000080000200004000000000080B0FDC6
:5C381000000000000000000000000000000000000000000001200000000010000000000000000000000000000000400000000000000000000000000000004000000000000000000000000000000040000000000000000000000000000000ECFE81
:5C386C0008000CC001000006000018000000000C4000300006000000000360800C8001300006000018000360000C0000000000000000C00000000060000C8001380006E00018000360000C0000300000000018000060000C00000000000089FCD3
:5C38C8000000B4800000000200000800000000B400001000020000000001A011048000100002000008000120000400000000000000004000000000200004801610005A40000800012000040000100000000008000020000400000000000094FF8B
:5C392400040000091601001811006001000000800800C00819200000002C0208300026C14418100060010C9021B00000000000000000000B0000008005320200C00200019360014C8011310200C00200000060000080113000000000008048FD56
:5C398000000038000700001C00007010000000380000E0001C000000000EC041380807E0001C000070100EC0013808000000000000008083000000C001380807E8001D880370400EC201380800E020000000701000C0413808000000000014FECC
:5C39DC00080030080600001800006000000000300000C00018000000000C8001310006C00018000060000C800130000000000000000000030000008001300006C00018040360000C8001300000C000000000600000800130000000000000C1FDCB
:5C3A38000000B0000600001800006000000000B00800C00018000000000C8009300006C00018000060000C800130000000000000000000030000008001300016C40018010360000C8001300000C00000000060000080013000000000000048FDD7
:5C3A940004000000000000000000000000000000000000000000000000000000000000000000000000000000000000000000000000000000000000000000000000000000000000000000000000000000000000000000000000000000008050FF03
:5C3AF000200004800010000240000800012000048000100002400008000120000480001000024000080001200004000000000010000240000800012000048000100002400008000120000480001000024000080001200004800010000200BCFC92
:5C3B4C00080000000000000000000000000000000000000000000000000000000000000000000000000000000000000000000000000000000000000000000000000000000000000000000000000000000000000000000000000000000000C5FE52
:5C3BA800200004800010000240000800012000048000100002400008000120000480001000024000080001200004000000000010000240000800012000048000100002400008000120000480001000024000080001200004800010000200BCFCD9
:5C3C040004002000048000100000400000000020000480001000020000080001200004800010000040000800012000000000000000000002000008000120000480001000024000080001200004800010000040000000012000000000008074FE7F
:5C3C600020000000000000004000000001200000000000000000000800000000000000000000400000000000000000000000001000020000080000000000000000000000000000000000000000000000400000000100000080001000020010FC46
:5C3CBC0008001000024000080000200000000010000240000800010000048000100002400008000020000480001000000000000000000001000004800010000240000800012000048000100002400008000020000080001000000000000075FC3E
:5C3D180020000000000000004000000001200000000000000000000800000000000000000000400000000000000000000000001000020000080000000000000000000000000000000000000000000000400000000100000080001000020010FC8D
:5C3D7400000000000000000000000000000000000000000000000000000000000000000000000000000000000000000000000000000000000000000000000000000000000000000000000000000000000000000000000000000000000000DCFF18
:5C3DD000000000000000000000000000000000000000000000000000000000000000000000000000000000000000000000000000000000000000000000000000000000000000000000000000000000000000000000000000000000000000DCFFBC
:5C3E2C00000000000000000000000000000000000000000000000000000000000000000000000000000000000000000000000000000000000000000000000000000000000000000000000000000000000000000000000000000000000000DCFF5F
:5C3E8800000000000000000000000000000000000000000000000000000000000000000000000000000000000000000000000000000000000000000000000000000000000000000000000000000000000000000000000000000000000000DCFF03
:5C3EE400000000000000000000000000000000000000000000000000000000240000000000000000000000000000000000000000000000000000000000000001000000400000000000000000000000000000000000000004000000000000E8FF32
:5C3F4000000000000000000000000000000000000000000000000000000000000000000000000000001000000000000000000000000000000000000000000000080020000000000000000000000000000000000000000000000000000000C4FC2D
:5C3F9C00000000000000000000000000000000000000000000000000000000000000000000000000000000000000000000000000000000000000000000000000000000000000000000000000000000000000000000000000000000000000DCFFEE
:5C3FF800000000000000000000000000000000000000000000000000000000000000000000000000000000000000000000000000000000000000000000000000000000000000000000000000000000000000000000000000000000000000DCFF92
:5C405400000000000000000000000000000000000000000000000000000000000000000000000000000000000000000000000000000000000000000000000000000000000000000000000000000000000000000000000000000000000000DCFF35
:5C40B000000000000000000000000000000000000000000000000000000000000000000000000000000000000000000000000000000000000000000000000000000000000000000000000000000000000000000000000000000000000000DCFFD9
:5C410C00000000000000000000000000000000000000000000000000000000000000000000000000000000000000000000000000000000000000000000000000000000000000000000000000000000000000000000000000000000000000DCFF7C
:5C416800000000020000000000000000000000200000000000000000000000000000000000000000000000000000000000000000000000000000000000000000000000000000000000000000000000000000000000000000000000000000DCFD00
:5C41C400000000000000000000000000000000000000000000000000000000000000000000000000000000000000000000000000000000000000000000000000000000000000000000000000000000000000000000000000000000000000DCFFC4
:5C422000000000000000000000000000000000000000000000000000000000000000000000000000000000000000000000000000000000000000000000000000000000000000000000000000000000000000000000000000000000000000DCFF67
:5C427C0000000000000120000000000000000000000010000000000000008000000000000000000000000400000000000000000000000000000000000000000200000000000000000040000000000000000000000000000000000000000054FF9C
:5C42D800000000000000000000000000000000000000000000000000000000000000000000000000000000000000000000000000000000000000000000000000000000000000000000000000000000000000000000000000000000000000DCFFAF
:5C43340000000000000240000000000000000000000020000000000000004000000000000000000000000200000000000000000000000000000000000000000100000000000000000080000500000000000000000000000000000000000038FFCC
:5C439000000000000000040000000000000000000000002000400000000000040100000000000000001000800010000000000000000000000010000000000010000000000100000080080001000000000000000000000000000000000000BCFD65
:5C43EC0000000000000000000000000000000000000000200000000000000000000000000000000000100020001000000000000000000000004000000000000000000000020000008000000000000000000000000000000000000000000000FF54
:5C444800000000000000000000000000000000000000000000000000000000000000000000000000000000000000000000000000000000000000000000000000000000000000000000000000000000000000000000000000000000000000DCFF3D
:5C44A400000000000000000000000000000000000000000000000000000000000000000000000000000000000000000000000000000000000000000000000000000000000000000000000000000000000000000000000000000000000000DCFFE1
:5C450000000000000000000000000000000000000000000000000000000000000000000000000000000000000000000000000000000000000000000000000000000000000000000000000000000000000000000000000000000000000000DCFF84
:5C455C00000000200000000000000000000000000000000000000000000000000000000000000000000000000000000000000000000000000000000000000000000000000000000000000000000000000000000000000000000000000000FCFFE8
:5C45B800000000000000000000000000000000000000000000000000000000100000000000000000000000000000000000000000000000000000000000000000000000000000040000000000000000000000000000000000000000000000C8FFCC
:5C461400000000000000000000000000000000000000000000000000000000000000000000000000000000000000000000000000000000000000000000000000000000000000000000000000000000000000000000000000000000000000DCFF6F
:5C467000000000000000000000000000000000000000000000000000000000000000000000000000000000000000000000000000000000000000000000000000000000000000000000000000000000000000000000000000000000000000DCFF13
:5C46CC00000000000000000000000000000000000000000000000000000000000000000000000000000000000000000000000000000000000000000000000000000000000000000000000000000000000000000000000000000000000000DCFFB7
:5C472800000000000000000000000000000000000000000000000000000000000000000000000000000000000000000000000000000000000000000000000000000000000000000000000000000000000000000000000000000000000000DCFF5A
:5C478400000000000000000000000000000000000000000000000000000000000000000000000000000000000000000000000000000000000000000000000000000000000000000000000000000000000000000000000000000000000000DCFFFE
:5C47E000000000000000000000001000000000000000000100000000000000000000000000000000000000000000000000000000000000000000000000000000000000000000000000000000000000000000000000000000000000000000CCFFA1
:5C483C00000000000000000000000000000000000000000000000000000000000000000000000000000000000000000000000000000000000000000000000000000000000000000000000000000000000000000000000000000000000000DCFF45
:5C489800000000000000000000000000000000000000000000000000000000000000000000000000000000000000000000000000000000000000000000000000000000000000000000000000000000000000000000000000000000000000DCFFE9
:5C48F40000000000000000000000000000000000000000000000000000000000000000000040000000000000000000000000000000000000000000000000000000000000000000000000000000000004000000000000000000000000000098FF8D
:5C495000000000000000000000000000000000000000000000000000000000000000004000000000000000000000000000000000000000000000000000000000000000000000000000000000000000000000000000000000000000000000D8FFF4
:5C49AC00000004000000000000000000000000000000000000000000000000000000B00000000000000000000080000000000000000000000000000000200A100000000010000010002040000000100000000000000050000100000000002CFD37
:5C4A08000000001000080000000000080000000000000020000000000000002002012000000000000000000000000000000000000000000000000000000000400000000080000020000400000000000100000018000020000000000000003CFF77
:5C4A640000000000000000010000000000000000000000000000000000000000000000000000000000000000000000000000000000000000000004008000000000000000000000000000000004000000000000000000000000000000000054FE1B
:5C4AC0000000000000000000000080000000000000000200000002000000000000080000000000000000002000000000000000000000000000000000000000000080000000000000000000000000000000000000000000000200000000007CFDF3
:5C4B1C00000000000000000000000000000000000000000000000000000000000000000000000000000000000000000000000000000000000000000000000000000000000000000000000000000000000000000000000000000000000000DCFF62
:5C4B7800000000000000000000000000000000000000000000000000000000000000000000000000000000000000000000000000000000000000000000000000000000000000000000000000000000000000000000000000000000000000DCFF06
:5C4BD400000020000000000000000000000000000000000000040000000000000000000000000000000000020000000000000000000000080000000000000000000020000000000000040000000000000000000000000000000000000000F4FD42
:5C4C300000000000000000000000000000000080040000000000000000000000000000000000000000000000000000000000000000000000000000000000800000000004000000000400000000000000000000000000000000000000000054FFC9
:5C4C8C001C0000000000000000000000000000000000000000000000000000000000000000000000000000000000000000000000000000000000000000000000000000000000000000000000000000000000000000000000000000000040B7FCBD
:5C4CE800000000000000000000000000000000000000000000000000000000000000000000000000000000000000000000000000000000000000000000000000000000000000000000000000000000000000000000000000000000000000DCFF95
:5C4D4400000000000001000000002000040000000000410004000022000000001000024080000000000004820000080000000000000000810010000000000000000000000100000080400000000000000000200004000010000000000000B4FFEE
:5C4DA000000000000000000000000000000000000000000000000000200000000000000000000000000000000000000000000000000040000000000000000000000000000000000100000000000000000000000000000000000000000000B8FEA0
:5C4DFC000000000000021400000A10000200000000A0220004000A114000000008000120400000000000024400A01000000000000000C0000120000000A000000000508000000001408000000000005000001000020000080000000000006CFFC2
:5C4E58000000140002000000000800103140020000000000000008A0010000009080080102020000200014820490000000000000000000010002008010C500000000480081200004004810084001202811050010248040100C000000000058FDA4
:5C4EB400000004800000000000000010000000000000000000000020000000001000000100000000200004220010000000000000000000010000008000000000000008008120000400401008000120080001001001804010080000000000FCFFF3
:5C4F1000000000000000000000000000000000000000000000000000000000000000000000000000000000000000000000000000000000000000000000000000000000000000000000000000000000000000000000000000100000000000CCFF6A
:5C4F6C0000000000000400000000004000000000200000800010000000000800012000040000000000400008000020000000000000000000020000000000200004000000000200000A00012000000000000000400000000120000000000098FD17
:5C4FC8001E00400000000000000000000000000000000000000000000000000000000000000000000000000000000000000000000000000000000000000000000000000000000000000000010000010000000000000000000000000000C05BFE14
:5C502400000000000000000000000010000000C003000000000000000008008020000000000000000000000000000000000000000000400000000000000080A000000000000000000000000000000000000000000000000800000000000070FDE0
:5C508000000000000000004000000000000000000000000000000000000000000000040000000000404000000000000000000000000000000000000000000000000000000000004000000004000000000000000000000000000000000000DCFFF1
:5C50DC00000000000000000000000000000000000000000000000000000000000000000000000000000000000000000000000000000000000000000000000000000000000000000000000000000000000000000000000000000000000000DCFF9D
:5C513800000000000000000000000000000000000000000000000000000000000000000000000000000000000000000000000000000000000000000000000000000000000000000000000000000000000000000000000000000000000000DCFF40
:5C519400000000000000000000000000000000000000000000000000000000000000000000000000000000000000000000000000000000000000000000000000000000000000000000000000000000000000000000000000000000000000DCFFE4
:5C51F000000000000000000000000000000000000000000000000000000000000000000000000000000000000000000000000000000000000000000000000000000000000000000000000000000000000000000000000000000000000000DCFF88
:5C524C0000000800000000000000000000000000000000010000000000002000000000000000000000000000000000000000000000000040000000000000000400004001000000020000000000008000000010000000000000000000000090FF37
:5C52A800000000080000000000000000000000000000000000000000000000008000000000000000000000000000000000000000000000000000000000000000000000000000000000000000000000000000000000000000000000000000DCFF47
:5C5304000000005000000000000000800000000050000000010000000000000002500008000000000080000000000000000000000000000004000000000040000A0000080004000010000240000000010000008000000002400000000000D8FD0E
:5C53600000000000000000000000000000000000000000000000000000008000000000000000000000000000000000000000000000000000000000000000000000000000000000000000000000000000000000000000000000000000000054FF1E
:5C53BC00000000000000008000100000000000000000000000400000004000000000000004800000080000000030020000000000000000000000000008000000000000000000000080110080000000000000000001000000002000000000D8FDB8
:5C54180000000000000000002000040000000000000000000000000000001000000000000001200000000000800040000000000000000000000000000002000000000000000000000000020000000000000000000000000000000800000040FFD8
:5C5474000000000000000006C0000000000000000000000000C0000400030000000000300006000018000060003C2000000000000000000000000060000000000000000000000000E00101800102000000000000030400008001000000008CFE6E
:5C54D000000000000000000240000000000000000000000000400B000001000000000010000200000800002000340100000000000000000000000020000000000000000000000000A009008046000000000000008D0000008000000000009CFD4E
:5C552C00000000000000009804230200000000000000000000001000008C0200000000C0041911006004008009300A00000000000000000000000080850000000000000000000000800500004004000000000000800000000006010000002CFC32
:5C558800000000000000001C80030000000000000000000000808300000E0000000000E0001C0000701000C0013900000000000000000000000000C0010000000000000000000000C041000007000000000000000E020000000700000000CCFEF7
:5C55E400000000000000001800030000000000000000000000000300000C0000000000C00018000060000080013000000000000000000000000000800100000000000000000000008001000006020000000000000C0200000006000000004CFDF1
:5C564000000000000000001800030000000000000000000000005300000C0000000000C00018000060000080013021000000000000000000000000800100000000000000000000008051000006000000000000002C00000000060000000018FFE9
:5C569C0004080000000000800000000000000000000000000000000002010000000000100080000008000080113002000000000000000000000000801100000000048000000000000000008000000000000000008C2000008000000000806CFD1E
:5C56F8000000020000000000200000000000000000000000000000018000000000000000000020000000000000024000000000000000000000000000000200000000012000000000000000000000000000000020001000000000000000000CFFF3
:5C575400680000000000000600000000000000000000000000C00018000300000000003040060000180000E0013C20000000000000000000000000E04100000030000600000000000000008001000000000018000F68000080010000000059FFA5
:5C57B00020000000000000020000000000000000000000000040000800010000000000D008020000080000A0513402000000000000000000000000A00500000010000200000000000000008000000000000008002D200000800000000000E4FE3B
:5C580C00840900000000009800000000000000000000000000001362142C000000000000021804006082008045B0200000000000000000000000008001000000C0241810000000000000000026000000000060042C80310000460100008014FE04
:5C586800C04100000000001C04000000000000000000000000800370000E0200000000E0001D0000700000C0013800000000000000000000000000C041000000E0001C00000000000000000007040000000070400EC40100000700000000A0FC2C
:5C58C400880100000000001800000000000000000000000000000360000C0000000000C020180000600000800132100000000000000000000000008001000000C0001800000000000000000006000000000060000C88010000060000000081FF83
:5C592000800100000000001800000000000000000000000000000360000C0000000000C0021800006000008009B0000000000000000000000000008081000000C0001800000000000000000006000000000060008C80010000060000000080FCE2
:5C597C0020000080000000800000000000000800800000040040006004010000000000000402000008000020003002000000000000000000000000000800000010000200100000000008040020000002000060040020000000200000008090FE14
:5C59D80000000000000000002000000000000002000000000100000080000000000000000001000000000000000040000000000000000000000000000002000000000000000400000000020000080000000000800004000000000800000058FE9D
:5C5A3400600000800100000600000000006000008001300000C0007800030000000000300006000018000060003C000000000000000000000000006000000000300006C00000000060000C80010000060000780003600000800100000000E5FF70
:5C5A90002800008000000002000000000020000080001000004000682001000000000010000200000800002000B410000000000000000000000000200000000010000240000000002000048000000002000068840120000080000000000000FEF6
:5C5AEC00808100004604005810000000008049000006C04400001360048C0100000000C0189800006002008005B0080000000000000000000000008011020000C0245800230200008051B04046010098040060048C80110000460000008020FFC7
:5C5B4800C00100000700001C0000000000C001000007E80000800371100E0000000000E0001C1000702000C0013900000000000000000000000000C001000000E0001C8803000000C00138000700001C000070100EC4410000070400000094FD32
:5C5BA400840100000600001800000000008001000006C00000000360400C0000000000C000180000600000800130000000000000000000000000008001000000C0001800030000008001300006000018000060100C800100000600000000A9FF4D
:5C5C0000800100000600001800000000008001000006C00000000360000C0000000000C0001800006000008001B0200000000000000000000000008001000000C0001800030000008001300006000018000060010C80010000060000000044FE09
:5C5C5C00240000000000000200000000000000008000C0080000230002400000000000C00880000000020000000400000000000000000000000000200000000000040200100000000008000120000002000008008C00080000460000000034FF55
:5C5CB80000000000000000000000000000000000000000000100000480001000000000000001200000800000800000000000000000000000000000000000000000000100000400000000024000080000000000000010000200000800000010FF62
:5C5D1400680000000000000600000000000000008001F00000C0031800030000000000F00006000018000060000C100000000000000000000000006000000000300006C00000000060000C8001000006000018200F60000080070000000004FF72
:5C5D7000200000000000000200000000000000008000D0220040830800010000000000D02402000008000020003402000000000000000000000000200000000010000240000000002000048000000002000068044D21000080260100000029FD64
:5C5DCC00840500000000001800000000000000000026C00800008B60100C0000000000C000980000600400805100000000000000000000000000000004000000C0025800630000008041B00046000058000000010C82110000160000000008FE0C
:5C5E2800C04100000000001C10000000000000000007E44000800370000E1000000000E0801C0800701000C00138080000000000000000000000004080000000E0201C8403000000C00138080701001C040070100EC04100000701000000D4FFBA
:5C5E8400880100000000001800000000000000000006C02000008360000C0000000000C000180000600000800130080000000000000000000000008081000000C0001800030000008001300006000018000060000C80010000060100008088FFB5
:5C5EE000800100000000001800000000000000000006C00800002360000C0000000000C022180000600000800130020000000000000000000000008011000000C0001800030000008001300006000018000060812C82010000460000000034FF1F
:5C5F3C00040800000000000200000000002000000020000400000008008C000000000010001801000002000000040000000000000002000000000080110000001000184100000000200000810000000200006004010008000020000000804CFEFE
:5C5F980000000200000000000000000000000000000008000100000100001000000000000000200000800000800000000000000000000000000000000002000000000020000000000000004000000000000000800000000200000800000038FE4F
:5C5FF400680000000000000600000000006000008001300000C00018000F000000000030401E000018000060000C00000000000000060000000000E00100000030001EC00000000060000C8001000006000078200360000080010000000045FE32
:5C605000200000000000000200000000002000008000100000400008004D0200000000D0081A040008000020000400000000000000020000000000A01101000010001A4400000000200004800000000200006802012000008000000000008CFE0C
:5C60AC00840500000000009800000000008051000026C00801000B60414C00000000000088980000600100801182000000000000001821000000008005000000C08858041300000080113022460100180300600020900500001600000080B8FD11
:5C610800C04100000000001C0400000000C001000007E10000808370000E0200000000E0001C0400701000C00108080000000000001C0000000000C041000000E0001C8003010000C00139000700001C0000704002C04100000702000000E8FF40
:5C616400880100000000001800000000008001000006C00000000360000C0200000000C020180000600000800130100000000000001800000000008001000000C0001804030000008001300006000018000060100C84010000060000000009FE18
:5C61C000800100000000001800000000008001000006C00000000360002C0000000000C004980400600000800130020000000000001800000000008005010000C0001800030000008001300006000018000060008C8001000006000000006CFD7D
:5C621C00240000000000001801000000000008000020100002000000024000000400001000800000080001000000010000000010000000000000000008000000C0088000230000000008008100000080000000000100080400200000008038FC62
:5C627800000000000000000020000000000000020000080000000001800010000000000000002000000000008000400000000000000000000000000000020000000001200004000000000240000000002000002000000002000008000000B8FCC8
:5C62D400680000000000001E00000000006000008001300007C00018000300000C0000304006000018000360000C000000000030000000000000006000000000F02006C08300000060000C8001020006000018000364000C80010000000035FECF
:5C633000200000000000009A04000000002000008000D0020240000800010000040000D008020000080001200004000000000010000000000000002000000000D0000240130000002000048046000002000008008D2000048000000000000CFD08
:5C638C00844100000000009800000000008051000016000458081360122C0000304200000859000060018C8405301200000000C0000000000000008005000000C00818000B000000804930000000009804006080408051300246000000800CFE19
:5C63E800C00100000000001C0800000000C001000007E1201C800374000E0200380000E0001C040070100EC041380000000000E080000000000000C001020000E0201CA083000000C00138200704001C000070000ED0013820070100000038FF01
:5C644400880100000000001808000000008001000006C02018000360000C0000300000C02018000060000C8001300000000000C0000000000000008001000000C0001800030000008001300006000018000060000C8201300006000000008DFF84
:5C64A000800100000000001801000000008001000006C00018000360000C0000300000C00818000060000C8001300000000000C0000000000000008001000000C0821800A30000008001300026010018000060008C8001300006000000000CFD31
:5C64FC00040800000000001801000000002000008000100000400008000120000001001000020000000200200000010000000000000000000000012000000000000480400000000120003082000000804000000001200000800000000080A8FC93
:5C65580000000200000000002000000000000000000000000000000000000000004000000000000000800000000040000000000000000000000000000000000000000120000000000000004000000000200000200000000000000000000084FDA3
:5C65B400680000000000001E00000000006000008001300001C00018000360000C0000300006000018000060000C000000000000000000000000036080000000300006C00000000360003C8801000006C00018000364000080010000000049FFE3
:5C661000200000000000001A04000000002000008000D0020040000800012000040000100002000008000020000400000000000000000000000001A01100000010000240000000012000B48000000002400008008D20000080000000000078FC8F
:5C666C00844100000000005800000000008005000026000200000B60102C8021B0080000841804006000008009310100000000000000000000000C0010000000C00458009300002C844930014600005800036041408011010006010000804CFE73
:5C66C800C00100000000001C0400000000C001020007E18000808370000EC80138000020001C0000701000C001382000000000000000000000000ED041000000E0801C840300000EC00138080701001C840374000EC2010000070000000068FE85
:5C672400880100000000001820000000008001000006C02000000360000C8001300000C0401800006000008001300000000000000000000000000C8001000000C00018000300000C8001300806000018000360000C8001000006000000000DFE5C
:5C678000800100000000009800000000008001000006C00400000360000C8001300000C0081800006000008001300000000000000000000000000C8051000000C00018000300000C8001300206000018000360004C8201000006000000003CFC43
:5C67DC0020000001001000020000080000200000800010000040000800010000048000100002400008000080110400000000000000004000000000200004000010008000100800002000048000000080000008000020000080001000020030FFA1
:5C683800000000400000000000000000000000000000000000000000000000000000000000000000000000000002000000000000000000000000000000000000000000200004000000000000000000002000000000040000000000000000F8FD85
:5C68940060000C000030000600001800006000008001300000C0001C000300000C9001304006C000180000E0010C1000000000000000C00000000060800C0000300006C00018000060000C8001020006000018200360000080013000060068FDB0
:5C68F000280004000010000200000800002000008000100000400B0800010000348200D008024000080000A0493402000000000000004000000000A011040000100002400008000020000480460000020000680401200000800010000200E1FFD1
:5C694C008009300600C0089804006004008049000016000200001061128C02000000160004980823610000800900020000000000000000230400000048300200C0029800936020008005B10040000098000000128C9005000026C20819205CFDDC
:5C69A800C041380000E0801C0000702000C001000007210001800370000E0000384007E8201C8003701000C0013A08000000000000008003000000C001384000E0201C8403700000C00138080704001C040070000EC041000007E0001C00ACFF92
:5C6A04008401300000C0001800006000008001000006C00001000360000C0000300006C020180003600000804130000000000000000000030000008001310000C0001800036000008001300006080018000060000C8001000006C000188074FE8C
:5C6A60008001300000C0001800006000008001000006C00200009360000C0000302206C0001800036000008011300A0000000000000000030000008009300000C0001800036000008001300046000018000060140C8001000006C0001800E0FE88
:5C6ABC0004000000000000000000000000000000000000000000000000000000000000000000000000000000000000000000000000000000000000000000000000000000000000000000000000000000000000000000000000000000008050FFAB
:5C6B1800200004800010000240000800012000048000100002400008000120000480001000024000080001200004000000000010000240000800012000048000100002400008000120000480001000024000080001200004800010000200BCFC39
:5C6B7400080000000000000000000000000000000000000000000000000000000000000000000000000000000000000000000000000000000000000000000000000000000000000000000000000000000000000000000000000000000000C5FEFA
:5C6BD000200004800010000240000800012000048000100002400008000120000480001000024000080001200004000000000010000240000800012000048000100002400008000120000480001000024000080001200004800010000200BCFC81
:5C6C2C00040120000480001000024000000001000004800010000240000800012000048000100002400008000120000000000080001000020000080001200000800010000240000800012000040000100002400008000120000480001080ACFD20
:5C6C880000000000000000000000000001000004000000000000000000000000000000000000000000000000000000000000000000000000080000000000800000000000000000000000000000100000000000000000000000000000000058FFBC
:5C6CE40088001000024000080001200000800000000240000800012000048000100002400008000120000480001000000000004000080001000004800010000040000800012000048000100002000008000120000480001000024000080099FD5A
:5C6D400000000000000000000000000001000004000000000000000000000000000000000000000000000000000000000000000000000000080000000000800000000000000000000000000000100000000000000000000000000000000058FF03
:5C6D9C00000000000000000000000000000000000000000000000000000000000000000000000000000000000000000000000000000000000000000000000000000000000000000000000000000000000000000000000000000000000000DCFFC0
:5C6DF800000000000000000000000000000000000000000000000000000000000000000000000000000000000000000000000000000000000000000000000000000000000000000000000000000000000000000000000000000000000000DCFF64
